Component: ARM Compiler 5.06 update 7 (build 960) Tool: armlink [4d3601]

==============================================================================

Section Cross References

    system_k1921vk035.o(i.SystemCoreClockUpdate) refers to system_k1921vk035.o(.data) for .data
    system_k1921vk035.o(i.SystemInit) refers to system_k1921vk035.o(i.ClkInit) for ClkInit
    system_k1921vk035.o(i.SystemInit) refers to system_k1921vk035.o(i.FPUInit) for FPUInit
    startup_k1921vk035.o(STACK) refers (Special) to heapauxi.o(.text) for __use_two_region_memory
    startup_k1921vk035.o(HEAP) refers (Special) to heapauxi.o(.text) for __use_two_region_memory
    startup_k1921vk035.o(RESET) refers (Special) to heapauxi.o(.text) for __use_two_region_memory
    startup_k1921vk035.o(RESET) refers to startup_k1921vk035.o(STACK) for __initial_sp
    startup_k1921vk035.o(RESET) refers to startup_k1921vk035.o(.text) for Reset_Handler
    startup_k1921vk035.o(RESET) refers to vk035_it.o(i.NMI_Handler) for NMI_Handler
    startup_k1921vk035.o(RESET) refers to vk035_it.o(i.HardFault_Handler) for HardFault_Handler
    startup_k1921vk035.o(RESET) refers to vk035_it.o(i.MemManage_Handler) for MemManage_Handler
    startup_k1921vk035.o(RESET) refers to vk035_it.o(i.BusFault_Handler) for BusFault_Handler
    startup_k1921vk035.o(RESET) refers to vk035_it.o(i.UsageFault_Handler) for UsageFault_Handler
    startup_k1921vk035.o(RESET) refers to vk035_it.o(i.SVC_Handler) for SVC_Handler
    startup_k1921vk035.o(RESET) refers to vk035_it.o(i.DebugMon_Handler) for DebugMon_Handler
    startup_k1921vk035.o(RESET) refers to vk035_it.o(i.PendSV_Handler) for PendSV_Handler
    startup_k1921vk035.o(RESET) refers to vk035_it.o(i.SysTick_Handler) for SysTick_Handler
    startup_k1921vk035.o(.text) refers (Special) to heapauxi.o(.text) for __use_two_region_memory
    startup_k1921vk035.o(.text) refers to system_k1921vk035.o(i.SystemInit) for SystemInit
    startup_k1921vk035.o(.text) refers to __main.o(!!!main) for __main
    startup_k1921vk035.o(.text) refers to startup_k1921vk035.o(HEAP) for Heap_Mem
    startup_k1921vk035.o(.text) refers to startup_k1921vk035.o(STACK) for Stack_Mem
    main.o(i.assert_failed) refers to _printf_percent.o(.ARM.Collect$$_printf_percent$$00000000) for _printf_percent
    main.o(i.assert_failed) refers to _printf_d.o(.ARM.Collect$$_printf_percent$$00000009) for _printf_d
    main.o(i.assert_failed) refers to _printf_s.o(.ARM.Collect$$_printf_percent$$00000014) for _printf_s
    main.o(i.assert_failed) refers to _printf_dec.o(.text) for _printf_int_dec
    main.o(i.assert_failed) refers to _printf_str.o(.text) for _printf_str
    main.o(i.assert_failed) refers to noretval__2printf.o(.text) for __2printf
    main.o(i.main) refers to main.o(i.periph_init) for periph_init
    main.o(i.periph_init) refers to _printf_pad.o(.text) for _printf_pre_padding
    main.o(i.periph_init) refers to _printf_percent.o(.ARM.Collect$$_printf_percent$$00000000) for _printf_percent
    main.o(i.periph_init) refers to _printf_d.o(.ARM.Collect$$_printf_percent$$00000009) for _printf_d
    main.o(i.periph_init) refers to _printf_dec.o(.text) for _printf_int_dec
    main.o(i.periph_init) refers to system_k1921vk035.o(i.SystemCoreClockUpdate) for SystemCoreClockUpdate
    main.o(i.periph_init) refers to rcu.o(i.sysclk_init) for sysclk_init
    main.o(i.periph_init) refers to gpio.o(i.gpio_init) for gpio_init
    main.o(i.periph_init) refers to retarget_conf.o(i.retarget_init) for retarget_init
    main.o(i.periph_init) refers to dflt_clz.o(x$fpl$dfltu) for __aeabi_ui2d
    main.o(i.periph_init) refers to ddiv.o(x$fpl$ddiv) for __aeabi_ddiv
    main.o(i.periph_init) refers to dfix.o(x$fpl$dfix) for __aeabi_d2iz
    main.o(i.periph_init) refers to noretval__2printf.o(.text) for __2printf
    main.o(i.periph_init) refers to system_k1921vk035.o(.data) for SystemCoreClock
    gpio.o(i.gpio_init) refers to plib035_gpio.o(i.GPIO_DeInit) for GPIO_DeInit
    gpio.o(i.gpio_init) refers to plib035_gpio.o(i.GPIO_Init) for GPIO_Init
    gpio.o(i.gpio_init) refers to gpio.o(.data) for .data
    rcu.o(i.RCU_ClkOutConfig) refers to main.o(i.assert_failed) for assert_failed
    rcu.o(i.sysclk_init) refers to plib035_rcu.o(i.RCU_PLL_AutoConfig) for RCU_PLL_AutoConfig
    rcu.o(i.sysclk_init) refers to main.o(i.Error_Handler) for Error_Handler
    rcu.o(i.sysclk_init) refers to system_k1921vk035.o(i.SystemCoreClockUpdate) for SystemCoreClockUpdate
    rcu.o(i.sysclk_init) refers to rcu.o(i.RCU_ClkOutConfig) for RCU_ClkOutConfig
    rcu.o(i.sysclk_init) refers to rcu.o(.data) for .data
    vk035_it.o(i.SysTick_Handler) refers to system_k1921vk035.o(.data) for uwTick
    plib035_adc.o(i.ADC_DC_Config) refers to main.o(i.assert_failed) for assert_failed
    plib035_adc.o(i.ADC_DC_Config) refers to plib035_adc.o(i.ADC_SEQ_Init) for i.ADC_SEQ_Init
    plib035_adc.o(i.ADC_DC_Init) refers to main.o(i.assert_failed) for assert_failed
    plib035_adc.o(i.ADC_DC_Init) refers to plib035_adc.o(i.ADC_DC_Config) for ADC_DC_Config
    plib035_adc.o(i.ADC_DC_Init) refers to plib035_adc.o(i.ADC_SEQ_Init) for i.ADC_SEQ_Init
    plib035_adc.o(i.ADC_DeInit) refers to plib035_adc.o(i.RCU_ADCRstCmd) for RCU_ADCRstCmd
    plib035_adc.o(i.ADC_SEQ_DCEnableCmd) refers to main.o(i.assert_failed) for assert_failed
    plib035_adc.o(i.ADC_SEQ_DCEnableCmd) refers to plib035_adc.o(i.ADC_SEQ_Init) for i.ADC_SEQ_Init
    plib035_adc.o(i.ADC_SEQ_Init) refers to main.o(i.assert_failed) for assert_failed
    plib035_adc.o(i.ADC_SEQ_Init) refers to plib035_adc.o(i.ADC_SEQ_ReqConfig) for ADC_SEQ_ReqConfig
    plib035_adc.o(i.ADC_SEQ_Init) refers to plib035_adc.o(i.ADC_SEQ_DCEnableCmd) for ADC_SEQ_DCEnableCmd
    plib035_adc.o(i.ADC_SEQ_ReqConfig) refers to main.o(i.assert_failed) for assert_failed
    plib035_adc.o(i.ADC_SEQ_ReqConfig) refers to plib035_adc.o(i.ADC_SEQ_Init) for i.ADC_SEQ_Init
    plib035_adc.o(i.RCU_ADCRstCmd) refers to main.o(i.assert_failed) for assert_failed
    plib035_dma.o(i.DMA_ChannelInit) refers to main.o(i.assert_failed) for assert_failed
    plib035_dma.o(i.DMA_Init) refers to plib035_dma.o(i.DMA_ProtectConfig) for DMA_ProtectConfig
    plib035_dma.o(i.DMA_Init) refers to main.o(i.assert_failed) for assert_failed
    plib035_dma.o(i.DMA_ProtectConfig) refers to main.o(i.assert_failed) for assert_failed
    plib035_dma.o(i.DMA_ProtectConfig) refers to plib035_dma.o(i.DMA_Init) for i.DMA_Init
    plib035_ecap.o(i.ECAP_Capture_Init) refers to main.o(i.assert_failed) for assert_failed
    plib035_ecap.o(i.ECAP_Capture_Init) refers to plib035_ecap.o(i.ECAP_Init) for i.ECAP_Init
    plib035_ecap.o(i.ECAP_DeInit) refers to main.o(i.assert_failed) for assert_failed
    plib035_ecap.o(i.ECAP_DeInit) refers to plib035_ecap.o(i.RCU_APBRstCmd) for RCU_APBRstCmd
    plib035_ecap.o(i.ECAP_Init) refers to main.o(i.assert_failed) for assert_failed
    plib035_ecap.o(i.ECAP_PWM_Init) refers to main.o(i.assert_failed) for assert_failed
    plib035_ecap.o(i.ECAP_PWM_Init) refers to plib035_ecap.o(i.ECAP_Init) for i.ECAP_Init
    plib035_ecap.o(i.RCU_APBRstCmd) refers to main.o(i.assert_failed) for assert_failed
    plib035_gpio.o(i.GPIO_AltFuncCmd) refers to main.o(i.assert_failed) for assert_failed
    plib035_gpio.o(i.GPIO_AltFuncCmd) refers to plib035_gpio.o(i.GPIO_DigitalCmd) for i.GPIO_DigitalCmd
    plib035_gpio.o(i.GPIO_DeInit) refers to main.o(i.assert_failed) for assert_failed
    plib035_gpio.o(i.GPIO_DeInit) refers to plib035_gpio.o(i.RCU_AHBRstCmd) for RCU_AHBRstCmd
    plib035_gpio.o(i.GPIO_DigitalCmd) refers to main.o(i.assert_failed) for assert_failed
    plib035_gpio.o(i.GPIO_DriveModeConfig) refers to main.o(i.assert_failed) for assert_failed
    plib035_gpio.o(i.GPIO_DriveModeConfig) refers to plib035_gpio.o(i.GPIO_ModeConfig) for GPIO_ModeConfig
    plib035_gpio.o(i.GPIO_InModeConfig) refers to main.o(i.assert_failed) for assert_failed
    plib035_gpio.o(i.GPIO_InModeConfig) refers to plib035_gpio.o(i.GPIO_ModeConfig) for GPIO_ModeConfig
    plib035_gpio.o(i.GPIO_Init) refers to plib035_gpio.o(i.GPIO_OutCmd) for GPIO_OutCmd
    plib035_gpio.o(i.GPIO_Init) refers to plib035_gpio.o(i.GPIO_AltFuncCmd) for GPIO_AltFuncCmd
    plib035_gpio.o(i.GPIO_Init) refers to plib035_gpio.o(i.GPIO_OutModeConfig) for GPIO_OutModeConfig
    plib035_gpio.o(i.GPIO_Init) refers to plib035_gpio.o(i.GPIO_InModeConfig) for GPIO_InModeConfig
    plib035_gpio.o(i.GPIO_Init) refers to plib035_gpio.o(i.GPIO_PullModeConfig) for GPIO_PullModeConfig
    plib035_gpio.o(i.GPIO_Init) refers to plib035_gpio.o(i.GPIO_DriveModeConfig) for GPIO_DriveModeConfig
    plib035_gpio.o(i.GPIO_Init) refers to plib035_gpio.o(i.GPIO_DigitalCmd) for GPIO_DigitalCmd
    plib035_gpio.o(i.GPIO_OutCmd) refers to main.o(i.assert_failed) for assert_failed
    plib035_gpio.o(i.GPIO_OutCmd) refers to plib035_gpio.o(i.GPIO_DigitalCmd) for i.GPIO_DigitalCmd
    plib035_gpio.o(i.GPIO_OutModeConfig) refers to main.o(i.assert_failed) for assert_failed
    plib035_gpio.o(i.GPIO_OutModeConfig) refers to plib035_gpio.o(i.GPIO_ModeConfig) for GPIO_ModeConfig
    plib035_gpio.o(i.GPIO_PullModeConfig) refers to main.o(i.assert_failed) for assert_failed
    plib035_gpio.o(i.GPIO_PullModeConfig) refers to plib035_gpio.o(i.GPIO_ModeConfig) for GPIO_ModeConfig
    plib035_gpio.o(i.RCU_AHBRstCmd) refers to main.o(i.assert_failed) for assert_failed
    plib035_i2c.o(i.I2C_FSFreqConfig) refers to main.o(i.assert_failed) for assert_failed
    plib035_i2c.o(i.I2C_HSFreqConfig) refers to main.o(i.assert_failed) for assert_failed
    plib035_i2c.o(i.I2C_HSFreqConfig) refers to plib035_i2c.o(i.I2C_FSFreqConfig) for i.I2C_FSFreqConfig
    plib035_mflash.o(i.MFLASH_EraseFull) refers to main.o(i.assert_failed) for assert_failed
    plib035_mflash.o(i.MFLASH_EraseFull) refers to plib035_mflash.o(i.MFLASH_SetCmd) for MFLASH_SetCmd
    plib035_mflash.o(i.MFLASH_EraseFull) refers to plib035_mflash.o(i.MFLASH_BusyStatus) for MFLASH_BusyStatus
    plib035_mflash.o(i.MFLASH_ErasePage) refers to main.o(i.assert_failed) for assert_failed
    plib035_mflash.o(i.MFLASH_ErasePage) refers to plib035_mflash.o(i.MFLASH_SetCmd) for MFLASH_SetCmd
    plib035_mflash.o(i.MFLASH_ErasePage) refers to plib035_mflash.o(i.MFLASH_BusyStatus) for MFLASH_BusyStatus
    plib035_mflash.o(i.MFLASH_ReadData) refers to main.o(i.assert_failed) for assert_failed
    plib035_mflash.o(i.MFLASH_ReadData) refers to plib035_mflash.o(i.MFLASH_SetCmd) for MFLASH_SetCmd
    plib035_mflash.o(i.MFLASH_ReadData) refers to plib035_mflash.o(i.MFLASH_BusyStatus) for MFLASH_BusyStatus
    plib035_mflash.o(i.MFLASH_WriteData) refers to main.o(i.assert_failed) for assert_failed
    plib035_mflash.o(i.MFLASH_WriteData) refers to plib035_mflash.o(i.MFLASH_SetCmd) for MFLASH_SetCmd
    plib035_mflash.o(i.MFLASH_WriteData) refers to plib035_mflash.o(i.MFLASH_BusyStatus) for MFLASH_BusyStatus
    plib035_mflash.o(i.MFLASH_WriteData) refers to plib035_mflash.o(i.MFLASH_ReadData) for i.MFLASH_ReadData
    plib035_pwm.o(i.PWM_AQ_ActionAConfig) refers to main.o(i.assert_failed) for assert_failed
    plib035_pwm.o(i.PWM_AQ_ActionBConfig) refers to main.o(i.assert_failed) for assert_failed
    plib035_pwm.o(i.PWM_AQ_Init) refers to plib035_pwm.o(i.PWM_AQ_ActionAConfig) for PWM_AQ_ActionAConfig
    plib035_pwm.o(i.PWM_AQ_Init) refers to plib035_pwm.o(i.PWM_AQ_ActionBConfig) for PWM_AQ_ActionBConfig
    plib035_pwm.o(i.PWM_CMP_CmpADirectLoadCmd) refers to main.o(i.assert_failed) for assert_failed
    plib035_pwm.o(i.PWM_CMP_CmpALoadEventConfig) refers to main.o(i.assert_failed) for assert_failed
    plib035_pwm.o(i.PWM_CMP_Init) refers to plib035_pwm.o(i.PWM_CMP_CmpALoadEventConfig) for PWM_CMP_CmpALoadEventConfig
    plib035_pwm.o(i.PWM_CMP_Init) refers to plib035_pwm.o(i.PWM_CMP_CmpADirectLoadCmd) for PWM_CMP_CmpADirectLoadCmd
    plib035_pwm.o(i.PWM_CMP_Init) refers to main.o(i.assert_failed) for assert_failed
    plib035_pwm.o(i.PWM_CMP_Init) refers to plib035_pwm.o(i.PWM_TB_Init) for i.PWM_TB_Init
    plib035_pwm.o(i.PWM_DB_Init) refers to main.o(i.assert_failed) for assert_failed
    plib035_pwm.o(i.PWM_DB_Init) refers to plib035_pwm.o(i.PWM_TB_Init) for i.PWM_TB_Init
    plib035_pwm.o(i.PWM_DeInit) refers to main.o(i.assert_failed) for assert_failed
    plib035_pwm.o(i.PWM_DeInit) refers to plib035_pwm.o(i.RCU_APBRstCmd) for RCU_APBRstCmd
    plib035_pwm.o(i.PWM_ET_Init) refers to main.o(i.assert_failed) for assert_failed
    plib035_pwm.o(i.PWM_ET_Init) refers to plib035_pwm.o(i.PWM_TB_Init) for i.PWM_TB_Init
    plib035_pwm.o(i.PWM_HD_Init) refers to main.o(i.assert_failed) for assert_failed
    plib035_pwm.o(i.PWM_HD_Init) refers to plib035_pwm.o(i.PWM_TB_Init) for i.PWM_TB_Init
    plib035_pwm.o(i.PWM_TB_ClkDivConfig) refers to main.o(i.assert_failed) for assert_failed
    plib035_pwm.o(i.PWM_TB_ClkDivConfig) refers to plib035_pwm.o(i.PWM_TB_Init) for i.PWM_TB_Init
    plib035_pwm.o(i.PWM_TB_Init) refers to main.o(i.assert_failed) for assert_failed
    plib035_pwm.o(i.PWM_TB_Init) refers to plib035_pwm.o(i.PWM_TB_ClkDivConfig) for PWM_TB_ClkDivConfig
    plib035_pwm.o(i.PWM_TZ_Init) refers to main.o(i.assert_failed) for assert_failed
    plib035_pwm.o(i.PWM_TZ_Init) refers to plib035_pwm.o(i.PWM_TB_Init) for i.PWM_TB_Init
    plib035_pwm.o(i.RCU_APBRstCmd) refers to main.o(i.assert_failed) for assert_failed
    plib035_qep.o(i.QEP_CAP_Init) refers to main.o(i.assert_failed) for assert_failed
    plib035_qep.o(i.QEP_CAP_Init) refers to plib035_qep.o(i.QEP_PC_Init) for i.QEP_PC_Init
    plib035_qep.o(i.QEP_CMP_Init) refers to main.o(i.assert_failed) for assert_failed
    plib035_qep.o(i.QEP_CMP_Init) refers to plib035_qep.o(i.QEP_PC_Init) for i.QEP_PC_Init
    plib035_qep.o(i.QEP_DeInit) refers to plib035_qep.o(i.RCU_APBRstCmd) for RCU_APBRstCmd
    plib035_qep.o(i.QEP_PC_Init) refers to main.o(i.assert_failed) for assert_failed
    plib035_qep.o(i.RCU_APBRstCmd) refers to main.o(i.assert_failed) for assert_failed
    plib035_rcu.o(i.MFLASH_LatencyConfig) refers to main.o(i.assert_failed) for assert_failed
    plib035_rcu.o(i.RCU_GetADCClkFreq) refers to plib035_rcu.o(i.getPeriphClkFreq) for getPeriphClkFreq
    plib035_rcu.o(i.RCU_GetClkOutFreq) refers to plib035_rcu.o(i.getSysPeriphClkFreq) for getSysPeriphClkFreq
    plib035_rcu.o(i.RCU_GetPLLDivClkFreq) refers to plib035_rcu.o(i.RCU_GetPLLClkFreq) for RCU_GetPLLClkFreq
    plib035_rcu.o(i.RCU_GetSPIClkFreq) refers to plib035_rcu.o(i.getPeriphClkFreq) for getPeriphClkFreq
    plib035_rcu.o(i.RCU_GetSysClkFreq) refers to plib035_rcu.o(i.getSysClkFreq) for getSysClkFreq
    plib035_rcu.o(i.RCU_GetTraceClkFreq) refers to plib035_rcu.o(i.getSysPeriphClkFreq) for getSysPeriphClkFreq
    plib035_rcu.o(i.RCU_GetUARTClkFreq) refers to plib035_rcu.o(i.getPeriphClkFreq) for getPeriphClkFreq
    plib035_rcu.o(i.RCU_GetWDTClkFreq) refers to plib035_rcu.o(i.getSysPeriphClkFreq) for getSysPeriphClkFreq
    plib035_rcu.o(i.RCU_PLL_AutoConfig) refers to plib035_rcu.o(i.RCU_PLL_StructInit) for RCU_PLL_StructInit
    plib035_rcu.o(i.RCU_PLL_AutoConfig) refers to plib035_rcu.o(i.RCU_PLL_Init) for RCU_PLL_Init
    plib035_rcu.o(i.RCU_PLL_AutoConfig) refers to plib035_rcu.o(i.MFLASH_LatencyConfig) for MFLASH_LatencyConfig
    plib035_rcu.o(i.RCU_PLL_AutoConfig) refers to plib035_rcu.o(i.RCU_SysClkChangeCmd) for RCU_SysClkChangeCmd
    plib035_rcu.o(i.RCU_PLL_DeInit) refers to plib035_rcu.o(i.RCU_PLL_OutCmd) for RCU_PLL_OutCmd
    plib035_rcu.o(i.RCU_PLL_Init) refers to main.o(i.assert_failed) for assert_failed
    plib035_rcu.o(i.RCU_PLL_Init) refers to plib035_rcu.o(i.RCU_PLL_OutCmd) for RCU_PLL_OutCmd
    plib035_rcu.o(i.RCU_PLL_OutCmd) refers to main.o(i.assert_failed) for assert_failed
    plib035_rcu.o(i.RCU_SysClkChangeCmd) refers to main.o(i.assert_failed) for assert_failed
    plib035_rcu.o(i.getPeriphClkFreq) refers to plib035_rcu.o(i.RCU_GetOSIClkFreq) for RCU_GetOSIClkFreq
    plib035_rcu.o(i.getPeriphClkFreq) refers to plib035_rcu.o(i.RCU_GetOSEClkFreq) for RCU_GetOSEClkFreq
    plib035_rcu.o(i.getPeriphClkFreq) refers to plib035_rcu.o(i.RCU_GetPLLClkFreq) for RCU_GetPLLClkFreq
    plib035_rcu.o(i.getPeriphClkFreq) refers to plib035_rcu.o(i.RCU_GetPLLDivClkFreq) for RCU_GetPLLDivClkFreq
    plib035_rcu.o(i.getSysClkFreq) refers to plib035_rcu.o(i.RCU_GetPLLDivClkFreq) for RCU_GetPLLDivClkFreq
    plib035_rcu.o(i.getSysClkFreq) refers to plib035_rcu.o(i.RCU_GetOSIClkFreq) for RCU_GetOSIClkFreq
    plib035_rcu.o(i.getSysClkFreq) refers to plib035_rcu.o(i.RCU_GetOSEClkFreq) for RCU_GetOSEClkFreq
    plib035_rcu.o(i.getSysClkFreq) refers to plib035_rcu.o(i.RCU_GetPLLClkFreq) for RCU_GetPLLClkFreq
    plib035_rcu.o(i.getSysPeriphClkFreq) refers to plib035_rcu.o(i.RCU_GetPLLDivClkFreq) for RCU_GetPLLDivClkFreq
    plib035_rcu.o(i.getSysPeriphClkFreq) refers to plib035_rcu.o(i.RCU_GetOSEClkFreq) for RCU_GetOSEClkFreq
    plib035_rcu.o(i.getSysPeriphClkFreq) refers to plib035_rcu.o(i.RCU_GetPLLClkFreq) for RCU_GetPLLClkFreq
    plib035_rcu.o(i.getSysPeriphClkFreq) refers to plib035_rcu.o(i.RCU_GetOSIClkFreq) for RCU_GetOSIClkFreq
    plib035_spi.o(i.RCU_SPIRstCmd) refers to main.o(i.assert_failed) for assert_failed
    plib035_spi.o(i.SPI_DeInit) refers to plib035_spi.o(i.RCU_SPIRstCmd) for RCU_SPIRstCmd
    plib035_spi.o(i.SPI_Init) refers to main.o(i.assert_failed) for assert_failed
    plib035_tmr.o(i.TMR_FreqConfig) refers to plib035_tmr.o(i.TMR_SetLoad) for TMR_SetLoad
    plib035_tmr.o(i.TMR_PeriodConfig) refers to plib035_tmr.o(i.TMR_SetLoad) for TMR_SetLoad
    plib035_tmr.o(i.TMR_SetLoad) refers to main.o(i.assert_failed) for assert_failed
    plib035_uart.o(i.RCU_UARTRstCmd) refers to main.o(i.assert_failed) for assert_failed
    plib035_uart.o(i.UART_AutoBaudConfig) refers to main.o(i.assert_failed) for assert_failed
    plib035_uart.o(i.UART_AutoBaudConfig) refers to plib035_rcu.o(i.RCU_GetUARTClkFreq) for RCU_GetUARTClkFreq
    plib035_uart.o(i.UART_DeInit) refers to main.o(i.assert_failed) for assert_failed
    plib035_uart.o(i.UART_DeInit) refers to plib035_uart.o(i.RCU_UARTRstCmd) for RCU_UARTRstCmd
    plib035_uart.o(i.UART_Init) refers to plib035_uart.o(i.UART_AutoBaudConfig) for UART_AutoBaudConfig
    plib035_uart.o(i.UART_Init) refers to main.o(i.assert_failed) for assert_failed
    retarget.o(.rev16_text) refers (Special) to use_no_semi.o(.text) for __use_no_semihosting_swi
    retarget.o(.revsh_text) refers (Special) to use_no_semi.o(.text) for __use_no_semihosting_swi
    retarget.o(.rrx_text) refers (Special) to use_no_semi.o(.text) for __use_no_semihosting_swi
    retarget.o(i._sys_exit) refers (Special) to use_no_semi.o(.text) for __use_no_semihosting_swi
    retarget.o(i._ttywrch) refers (Special) to use_no_semi.o(.text) for __use_no_semihosting_swi
    retarget.o(i._ttywrch) refers to retarget_conf.o(i.retarget_put_char) for retarget_put_char
    retarget.o(i.ferror) refers (Special) to use_no_semi.o(.text) for __use_no_semihosting_swi
    retarget.o(i.fgetc) refers (Special) to use_no_semi.o(.text) for __use_no_semihosting_swi
    retarget.o(i.fgetc) refers to retarget_conf.o(i.retarget_get_char) for retarget_get_char
    retarget.o(i.fputc) refers (Special) to use_no_semi.o(.text) for __use_no_semihosting_swi
    retarget.o(i.fputc) refers to retarget_conf.o(i.retarget_put_char) for retarget_put_char
    retarget.o(.data) refers (Special) to use_no_semi.o(.text) for __use_no_semihosting_swi
    retarget.o(.data) refers (Special) to use_no_semi.o(.text) for __use_no_semihosting_swi
    retarget_conf.o(i.retarget_init) refers to system_k1921vk035.o(.data) for SystemCoreClock
    __2printf.o(.text) refers to _printf_char_file.o(.text) for _printf_char_file
    __2printf.o(.text) refers to retarget.o(.data) for __stdout
    noretval__2printf.o(.text) refers to _printf_char_file.o(.text) for _printf_char_file
    noretval__2printf.o(.text) refers to retarget.o(.data) for __stdout
    __printf.o(.text) refers to _printf_percent.o(.ARM.Collect$$_printf_percent$$00000000) for _printf_percent
    _printf_str.o(.text) refers (Special) to _printf_char.o(.text) for _printf_cs_common
    _printf_str.o(.text) refers (Weak) to _printf_pad.o(.text) for _printf_pre_padding
    _printf_str.o(.text) refers (Weak) to _printf_pad.o(.text) for _printf_post_padding
    _printf_dec.o(.text) refers to _printf_intcommon.o(.text) for _printf_int_common
    __printf_flags.o(.text) refers to _printf_percent.o(.ARM.Collect$$_printf_percent$$00000000) for _printf_percent
    __printf_flags.o(.text) refers to __printf_flags.o(.constdata) for .constdata
    __printf_ss.o(.text) refers to _printf_percent.o(.ARM.Collect$$_printf_percent$$00000000) for _printf_percent
    __printf_flags_ss.o(.text) refers to _printf_percent.o(.ARM.Collect$$_printf_percent$$00000000) for _printf_percent
    __printf_flags_ss.o(.text) refers to __printf_flags_ss.o(.constdata) for .constdata
    __printf_wp.o(.text) refers to __printf_wp.o(i._is_digit) for _is_digit
    __printf_wp.o(.text) refers to _printf_percent.o(.ARM.Collect$$_printf_percent$$00000000) for _printf_percent
    __printf_flags_wp.o(.text) refers to __printf_wp.o(i._is_digit) for _is_digit
    __printf_flags_wp.o(.text) refers to _printf_percent.o(.ARM.Collect$$_printf_percent$$00000000) for _printf_percent
    __printf_flags_wp.o(.text) refers to __printf_flags_wp.o(.constdata) for .constdata
    __printf_ss_wp.o(.text) refers to __printf_wp.o(i._is_digit) for _is_digit
    __printf_ss_wp.o(.text) refers to _printf_percent.o(.ARM.Collect$$_printf_percent$$00000000) for _printf_percent
    __printf_flags_ss_wp.o(.text) refers to __printf_wp.o(i._is_digit) for _is_digit
    __printf_flags_ss_wp.o(.text) refers to _printf_percent.o(.ARM.Collect$$_printf_percent$$00000000) for _printf_percent
    __printf_flags_ss_wp.o(.text) refers to __printf_flags_ss_wp.o(.constdata) for .constdata
    _printf_s.o(.ARM.Collect$$_printf_percent$$00000014) refers (Weak) to _printf_char.o(.text) for _printf_string
    _printf_d.o(.ARM.Collect$$_printf_percent$$00000009) refers (Weak) to _printf_dec.o(.text) for _printf_int_dec
    _printf_percent.o(.ARM.Collect$$_printf_percent$$00000000) refers (Special) to _printf_percent_end.o(.ARM.Collect$$_printf_percent$$00000017) for _printf_percent_end
    __main.o(!!!main) refers to __rtentry.o(.ARM.Collect$$rtentry$$00000000) for __rt_entry
    ddiv.o(x$fpl$drdiv) refers (Special) to usenofp.o(x$fpl$usenofp) for __I$use$fp
    ddiv.o(x$fpl$drdiv) refers to ddiv.o(x$fpl$ddiv) for ddiv_entry
    ddiv.o(x$fpl$ddiv) refers (Special) to usenofp.o(x$fpl$usenofp) for __I$use$fp
    ddiv.o(x$fpl$ddiv) refers to dretinf.o(x$fpl$dretinf) for __fpl_dretinf
    ddiv.o(x$fpl$ddiv) refers to dnaninf.o(x$fpl$dnaninf) for __fpl_dnaninf
    dfix.o(x$fpl$dfix) refers (Special) to usenofp.o(x$fpl$usenofp) for __I$use$fp
    dfix.o(x$fpl$dfix) refers to dnaninf.o(x$fpl$dnaninf) for __fpl_dnaninf
    dfix.o(x$fpl$dfixr) refers (Special) to usenofp.o(x$fpl$usenofp) for __I$use$fp
    dfix.o(x$fpl$dfixr) refers to dnaninf.o(x$fpl$dnaninf) for __fpl_dnaninf
    dflt_clz.o(x$fpl$dfltu) refers (Special) to usenofp.o(x$fpl$usenofp) for __I$use$fp
    dflt_clz.o(x$fpl$dflt) refers (Special) to usenofp.o(x$fpl$usenofp) for __I$use$fp
    dflt_clz.o(x$fpl$dfltn) refers (Special) to usenofp.o(x$fpl$usenofp) for __I$use$fp
    __rtentry.o(.ARM.Collect$$rtentry$$00000000) refers (Special) to __rtentry2.o(.ARM.Collect$$rtentry$$0000000A) for __rt_entry_li
    __rtentry.o(.ARM.Collect$$rtentry$$00000000) refers (Special) to __rtentry2.o(.ARM.Collect$$rtentry$$0000000D) for __rt_entry_main
    __rtentry.o(.ARM.Collect$$rtentry$$00000000) refers (Special) to __rtentry2.o(.ARM.Collect$$rtentry$$0000000C) for __rt_entry_postli_1
    __rtentry.o(.ARM.Collect$$rtentry$$00000000) refers (Special) to __rtentry2.o(.ARM.Collect$$rtentry$$00000009) for __rt_entry_postsh_1
    __rtentry.o(.ARM.Collect$$rtentry$$00000000) refers (Special) to __rtentry2.o(.ARM.Collect$$rtentry$$00000002) for __rt_entry_presh_1
    __rtentry.o(.ARM.Collect$$rtentry$$00000000) refers (Special) to __rtentry4.o(.ARM.Collect$$rtentry$$00000004) for __rt_entry_sh
    _printf_intcommon.o(.text) refers (Weak) to _printf_pad.o(.text) for _printf_pre_padding
    _printf_intcommon.o(.text) refers (Weak) to _printf_pad.o(.text) for _printf_pre_padding
    _printf_intcommon.o(.text) refers (Weak) to _printf_pad.o(.text) for _printf_post_padding
    _printf_char.o(.text) refers (Weak) to _printf_str.o(.text) for _printf_str
    _printf_char_file.o(.text) refers to _printf_char_common.o(.text) for _printf_char_common
    _printf_char_file.o(.text) refers to retarget.o(i.ferror) for ferror
    _printf_char_file.o(.text) refers to retarget.o(i.fputc) for fputc
    dnaninf.o(x$fpl$dnaninf) refers (Special) to usenofp.o(x$fpl$usenofp) for __I$use$fp
    dretinf.o(x$fpl$dretinf) refers (Special) to usenofp.o(x$fpl$usenofp) for __I$use$fp
    __rtentry2.o(.ARM.Collect$$rtentry$$00000008) refers to boardinit2.o(.text) for _platform_post_stackheap_init
    __rtentry2.o(.ARM.Collect$$rtentry$$0000000A) refers to libinit.o(.ARM.Collect$$libinit$$00000000) for __rt_lib_init
    __rtentry2.o(.ARM.Collect$$rtentry$$0000000B) refers to boardinit3.o(.text) for _platform_post_lib_init
    __rtentry2.o(.ARM.Collect$$rtentry$$0000000D) refers to main.o(i.main) for main
    __rtentry2.o(.ARM.Collect$$rtentry$$0000000D) refers to exit.o(.text) for exit
    __rtentry2.o(.ARM.exidx) refers to __rtentry2.o(.ARM.Collect$$rtentry$$00000001) for .ARM.Collect$$rtentry$$00000001
    __rtentry2.o(.ARM.exidx) refers to __rtentry2.o(.ARM.Collect$$rtentry$$00000008) for .ARM.Collect$$rtentry$$00000008
    __rtentry2.o(.ARM.exidx) refers to __rtentry2.o(.ARM.Collect$$rtentry$$0000000A) for .ARM.Collect$$rtentry$$0000000A
    __rtentry2.o(.ARM.exidx) refers to __rtentry2.o(.ARM.Collect$$rtentry$$0000000B) for .ARM.Collect$$rtentry$$0000000B
    __rtentry2.o(.ARM.exidx) refers to __rtentry2.o(.ARM.Collect$$rtentry$$0000000D) for .ARM.Collect$$rtentry$$0000000D
    __rtentry4.o(.ARM.Collect$$rtentry$$00000004) refers to sys_stackheap_outer.o(.text) for __user_setup_stackheap
    __rtentry4.o(.ARM.exidx) refers to __rtentry4.o(.ARM.Collect$$rtentry$$00000004) for .ARM.Collect$$rtentry$$00000004
    _printf_char_common.o(.text) refers to __printf_wp.o(.text) for __printf
    sys_stackheap_outer.o(.text) refers to libspace.o(.text) for __user_perproc_libspace
    sys_stackheap_outer.o(.text) refers to startup_k1921vk035.o(.text) for __user_initial_stackheap
    exit.o(.text) refers to rtexit.o(.ARM.Collect$$rtexit$$00000000) for __rt_exit
    libinit.o(.ARM.Collect$$libinit$$00000000) refers (Special) to libinit2.o(.ARM.Collect$$libinit$$0000002E) for __rt_lib_init_alloca_1
    libinit.o(.ARM.Collect$$libinit$$00000000) refers (Special) to libinit2.o(.ARM.Collect$$libinit$$0000002C) for __rt_lib_init_argv_1
    libinit.o(.ARM.Collect$$libinit$$00000000) refers (Special) to libinit2.o(.ARM.Collect$$libinit$$0000001B) for __rt_lib_init_atexit_1
    libinit.o(.ARM.Collect$$libinit$$00000000) refers (Special) to libinit2.o(.ARM.Collect$$libinit$$00000021) for __rt_lib_init_clock_1
    libinit.o(.ARM.Collect$$libinit$$00000000) refers (Special) to libinit2.o(.ARM.Collect$$libinit$$00000032) for __rt_lib_init_cpp_1
    libinit.o(.ARM.Collect$$libinit$$00000000) refers (Special) to libinit2.o(.ARM.Collect$$libinit$$00000030) for __rt_lib_init_exceptions_1
    libinit.o(.ARM.Collect$$libinit$$00000000) refers (Special) to libinit2.o(.ARM.Collect$$libinit$$00000001) for __rt_lib_init_fp_1
    libinit.o(.ARM.Collect$$libinit$$00000000) refers (Special) to libinit2.o(.ARM.Collect$$libinit$$0000001F) for __rt_lib_init_fp_trap_1
    libinit.o(.ARM.Collect$$libinit$$00000000) refers (Special) to libinit2.o(.ARM.Collect$$libinit$$00000023) for __rt_lib_init_getenv_1
    libinit.o(.ARM.Collect$$libinit$$00000000) refers (Special) to libinit2.o(.ARM.Collect$$libinit$$0000000A) for __rt_lib_init_heap_1
    libinit.o(.ARM.Collect$$libinit$$00000000) refers (Special) to libinit2.o(.ARM.Collect$$libinit$$00000011) for __rt_lib_init_lc_collate_1
    libinit.o(.ARM.Collect$$libinit$$00000000) refers (Special) to libinit2.o(.ARM.Collect$$libinit$$00000013) for __rt_lib_init_lc_ctype_1
    libinit.o(.ARM.Collect$$libinit$$00000000) refers (Special) to libinit2.o(.ARM.Collect$$libinit$$00000015) for __rt_lib_init_lc_monetary_1
    libinit.o(.ARM.Collect$$libinit$$00000000) refers (Special) to libinit2.o(.ARM.Collect$$libinit$$00000017) for __rt_lib_init_lc_numeric_1
    libinit.o(.ARM.Collect$$libinit$$00000000) refers (Special) to libinit2.o(.ARM.Collect$$libinit$$00000019) for __rt_lib_init_lc_time_1
    libinit.o(.ARM.Collect$$libinit$$00000000) refers (Special) to libinit2.o(.ARM.Collect$$libinit$$00000004) for __rt_lib_init_preinit_1
    libinit.o(.ARM.Collect$$libinit$$00000000) refers (Special) to libinit2.o(.ARM.Collect$$libinit$$0000000E) for __rt_lib_init_rand_1
    libinit.o(.ARM.Collect$$libinit$$00000000) refers (Special) to libinit2.o(.ARM.Collect$$libinit$$00000033) for __rt_lib_init_return
    libinit.o(.ARM.Collect$$libinit$$00000000) refers (Special) to libinit2.o(.ARM.Collect$$libinit$$0000001D) for __rt_lib_init_signal_1
    libinit.o(.ARM.Collect$$libinit$$00000000) refers (Special) to libinit2.o(.ARM.Collect$$libinit$$00000025) for __rt_lib_init_stdio_1
    libinit.o(.ARM.Collect$$libinit$$00000000) refers (Special) to libinit2.o(.ARM.Collect$$libinit$$0000000C) for __rt_lib_init_user_alloc_1
    libspace.o(.text) refers to libspace.o(.bss) for __libspace_start
    rtexit.o(.ARM.Collect$$rtexit$$00000000) refers (Special) to rtexit2.o(.ARM.Collect$$rtexit$$00000004) for __rt_exit_exit
    rtexit.o(.ARM.Collect$$rtexit$$00000000) refers (Special) to rtexit2.o(.ARM.Collect$$rtexit$$00000003) for __rt_exit_ls
    rtexit.o(.ARM.Collect$$rtexit$$00000000) refers (Special) to rtexit2.o(.ARM.Collect$$rtexit$$00000002) for __rt_exit_prels_1
    rtexit.o(.ARM.exidx) refers (Special) to rtexit2.o(.ARM.Collect$$rtexit$$00000004) for __rt_exit_exit
    rtexit.o(.ARM.exidx) refers (Special) to rtexit2.o(.ARM.Collect$$rtexit$$00000003) for __rt_exit_ls
    rtexit.o(.ARM.exidx) refers (Special) to rtexit2.o(.ARM.Collect$$rtexit$$00000002) for __rt_exit_prels_1
    rtexit.o(.ARM.exidx) refers to rtexit.o(.ARM.Collect$$rtexit$$00000000) for .ARM.Collect$$rtexit$$00000000
    libinit2.o(.ARM.Collect$$libinit$$00000001) refers to fpinit.o(x$fpl$fpinit) for _fp_init
    libinit2.o(.ARM.Collect$$libinit$$00000010) refers to libinit2.o(.ARM.Collect$$libinit$$0000000F) for .ARM.Collect$$libinit$$0000000F
    libinit2.o(.ARM.Collect$$libinit$$00000012) refers to libinit2.o(.ARM.Collect$$libinit$$0000000F) for .ARM.Collect$$libinit$$0000000F
    libinit2.o(.ARM.Collect$$libinit$$00000014) refers to libinit2.o(.ARM.Collect$$libinit$$0000000F) for .ARM.Collect$$libinit$$0000000F
    libinit2.o(.ARM.Collect$$libinit$$00000016) refers to libinit2.o(.ARM.Collect$$libinit$$0000000F) for .ARM.Collect$$libinit$$0000000F
    libinit2.o(.ARM.Collect$$libinit$$00000018) refers to libinit2.o(.ARM.Collect$$libinit$$0000000F) for .ARM.Collect$$libinit$$0000000F
    libinit2.o(.ARM.Collect$$libinit$$00000026) refers to argv_veneer.o(.emb_text) for __ARM_argv_veneer
    libinit2.o(.ARM.Collect$$libinit$$00000027) refers to argv_veneer.o(.emb_text) for __ARM_argv_veneer
    rtexit2.o(.ARM.Collect$$rtexit$$00000003) refers to libshutdown.o(.ARM.Collect$$libshutdown$$00000000) for __rt_lib_shutdown
    rtexit2.o(.ARM.Collect$$rtexit$$00000004) refers to retarget.o(i._sys_exit) for _sys_exit
    rtexit2.o(.ARM.exidx) refers to rtexit2.o(.ARM.Collect$$rtexit$$00000001) for .ARM.Collect$$rtexit$$00000001
    rtexit2.o(.ARM.exidx) refers to rtexit2.o(.ARM.Collect$$rtexit$$00000003) for .ARM.Collect$$rtexit$$00000003
    rtexit2.o(.ARM.exidx) refers to rtexit2.o(.ARM.Collect$$rtexit$$00000004) for .ARM.Collect$$rtexit$$00000004
    argv_veneer.o(.emb_text) refers to no_argv.o(.text) for __ARM_get_argv
    _get_argv_nomalloc.o(.text) refers (Special) to hrguard.o(.text) for __heap_region$guard
    _get_argv_nomalloc.o(.text) refers to defsig_rtmem_outer.o(.text) for __rt_SIGRTMEM
    _get_argv_nomalloc.o(.text) refers to sys_command.o(.text) for _sys_command_string
    libshutdown.o(.ARM.Collect$$libshutdown$$00000000) refers (Special) to libshutdown2.o(.ARM.Collect$$libshutdown$$00000004) for __rt_lib_shutdown_cpp_1
    libshutdown.o(.ARM.Collect$$libshutdown$$00000000) refers (Special) to libshutdown2.o(.ARM.Collect$$libshutdown$$00000002) for __rt_lib_shutdown_fini_1
    libshutdown.o(.ARM.Collect$$libshutdown$$00000000) refers (Special) to libshutdown2.o(.ARM.Collect$$libshutdown$$00000009) for __rt_lib_shutdown_fp_trap_1
    libshutdown.o(.ARM.Collect$$libshutdown$$00000000) refers (Special) to libshutdown2.o(.ARM.Collect$$libshutdown$$00000011) for __rt_lib_shutdown_heap_1
    libshutdown.o(.ARM.Collect$$libshutdown$$00000000) refers (Special) to libshutdown2.o(.ARM.Collect$$libshutdown$$00000012) for __rt_lib_shutdown_return
    libshutdown.o(.ARM.Collect$$libshutdown$$00000000) refers (Special) to libshutdown2.o(.ARM.Collect$$libshutdown$$0000000C) for __rt_lib_shutdown_signal_1
    libshutdown.o(.ARM.Collect$$libshutdown$$00000000) refers (Special) to libshutdown2.o(.ARM.Collect$$libshutdown$$00000006) for __rt_lib_shutdown_stdio_1
    libshutdown.o(.ARM.Collect$$libshutdown$$00000000) refers (Special) to libshutdown2.o(.ARM.Collect$$libshutdown$$0000000E) for __rt_lib_shutdown_user_alloc_1
    sys_command.o(.text) refers (Special) to use_no_semi.o(.text) for __I$use$semihosting
    sys_command.o(.text) refers (Special) to indicate_semi.o(.text) for __semihosting_library_function
    defsig_rtmem_outer.o(.text) refers to defsig_rtmem_inner.o(.text) for __rt_SIGRTMEM_inner
    defsig_rtmem_outer.o(.text) refers to defsig_exit.o(.text) for __sig_exit
    defsig_rtmem_formal.o(.text) refers to rt_raise.o(.text) for __rt_raise
    rt_raise.o(.text) refers to __raise.o(.text) for __raise
    rt_raise.o(.text) refers to retarget.o(i._sys_exit) for _sys_exit
    defsig_exit.o(.text) refers to retarget.o(i._sys_exit) for _sys_exit
    defsig_rtmem_inner.o(.text) refers to defsig_general.o(.text) for __default_signal_display
    __raise.o(.text) refers to defsig.o(CL$$defsig) for __default_signal_handler
    defsig_general.o(.text) refers to retarget.o(i._ttywrch) for _ttywrch
    defsig.o(CL$$defsig) refers to defsig_rtmem_inner.o(.text) for __rt_SIGRTMEM_inner
    defsig_abrt_inner.o(.text) refers to defsig_general.o(.text) for __default_signal_display
    defsig_fpe_inner.o(.text) refers to defsig_general.o(.text) for __default_signal_display
    defsig_rtred_inner.o(.text) refers to defsig_general.o(.text) for __default_signal_display
    defsig_stak_inner.o(.text) refers to defsig_general.o(.text) for __default_signal_display
    defsig_pvfn_inner.o(.text) refers to defsig_general.o(.text) for __default_signal_display
    defsig_cppl_inner.o(.text) refers to defsig_general.o(.text) for __default_signal_display
    defsig_segv_inner.o(.text) refers to defsig_general.o(.text) for __default_signal_display
    defsig_other.o(.text) refers to defsig_general.o(.text) for __default_signal_display


==============================================================================

Removing Unused input sections from the image.

    Removing system_k1921vk035.o(.rev16_text), (4 bytes).
    Removing system_k1921vk035.o(.revsh_text), (4 bytes).
    Removing system_k1921vk035.o(.rrx_text), (6 bytes).
    Removing main.o(.rev16_text), (4 bytes).
    Removing main.o(.revsh_text), (4 bytes).
    Removing main.o(.rrx_text), (6 bytes).
    Removing gpio.o(.rev16_text), (4 bytes).
    Removing gpio.o(.revsh_text), (4 bytes).
    Removing gpio.o(.rrx_text), (6 bytes).
    Removing rcu.o(.rev16_text), (4 bytes).
    Removing rcu.o(.revsh_text), (4 bytes).
    Removing rcu.o(.rrx_text), (6 bytes).
    Removing vk035_it.o(.rev16_text), (4 bytes).
    Removing vk035_it.o(.revsh_text), (4 bytes).
    Removing vk035_it.o(.rrx_text), (6 bytes).
    Removing plib035_adc.o(.rev16_text), (4 bytes).
    Removing plib035_adc.o(.revsh_text), (4 bytes).
    Removing plib035_adc.o(.rrx_text), (6 bytes).
    Removing plib035_adc.o(i.ADC_DC_Config), (116 bytes).
    Removing plib035_adc.o(i.ADC_DC_Init), (316 bytes).
    Removing plib035_adc.o(i.ADC_DC_StructInit), (18 bytes).
    Removing plib035_adc.o(i.ADC_DeInit), (18 bytes).
    Removing plib035_adc.o(i.ADC_SEQ_DCEnableCmd), (96 bytes).
    Removing plib035_adc.o(i.ADC_SEQ_Init), (568 bytes).
    Removing plib035_adc.o(i.ADC_SEQ_ReqConfig), (104 bytes).
    Removing plib035_adc.o(i.ADC_SEQ_StructInit), (52 bytes).
    Removing plib035_adc.o(i.RCU_ADCRstCmd), (80 bytes).
    Removing plib035_can.o(.rev16_text), (4 bytes).
    Removing plib035_can.o(.revsh_text), (4 bytes).
    Removing plib035_can.o(.rrx_text), (6 bytes).
    Removing plib035_dma.o(.rev16_text), (4 bytes).
    Removing plib035_dma.o(.revsh_text), (4 bytes).
    Removing plib035_dma.o(.rrx_text), (6 bytes).
    Removing plib035_dma.o(i.DMA_ChannelDeInit), (10 bytes).
    Removing plib035_dma.o(i.DMA_ChannelInit), (492 bytes).
    Removing plib035_dma.o(i.DMA_ChannelStructInit), (40 bytes).
    Removing plib035_dma.o(i.DMA_DeInit), (28 bytes).
    Removing plib035_dma.o(i.DMA_Init), (292 bytes).
    Removing plib035_dma.o(i.DMA_ProtectConfig), (100 bytes).
    Removing plib035_dma.o(i.DMA_StructInit), (26 bytes).
    Removing plib035_ecap.o(.rev16_text), (4 bytes).
    Removing plib035_ecap.o(.revsh_text), (4 bytes).
    Removing plib035_ecap.o(.rrx_text), (6 bytes).
    Removing plib035_ecap.o(i.ECAP_Capture_Init), (632 bytes).
    Removing plib035_ecap.o(i.ECAP_Capture_StructInit), (28 bytes).
    Removing plib035_ecap.o(i.ECAP_DeInit), (124 bytes).
    Removing plib035_ecap.o(i.ECAP_Init), (276 bytes).
    Removing plib035_ecap.o(i.ECAP_PWM_Init), (144 bytes).
    Removing plib035_ecap.o(i.ECAP_PWM_StructInit), (18 bytes).
    Removing plib035_ecap.o(i.ECAP_StructInit), (12 bytes).
    Removing plib035_ecap.o(i.RCU_APBRstCmd), (152 bytes).
    Removing plib035_gpio.o(.rev16_text), (4 bytes).
    Removing plib035_gpio.o(.revsh_text), (4 bytes).
    Removing plib035_gpio.o(.rrx_text), (6 bytes).
    Removing plib035_gpio.o(i.GPIO_StructInit), (24 bytes).
    Removing plib035_i2c.o(.rev16_text), (4 bytes).
    Removing plib035_i2c.o(.revsh_text), (4 bytes).
    Removing plib035_i2c.o(.rrx_text), (6 bytes).
    Removing plib035_i2c.o(i.I2C_FSFreqConfig), (104 bytes).
    Removing plib035_i2c.o(i.I2C_HSFreqConfig), (72 bytes).
    Removing plib035_mflash.o(.rev16_text), (4 bytes).
    Removing plib035_mflash.o(.revsh_text), (4 bytes).
    Removing plib035_mflash.o(.rrx_text), (6 bytes).
    Removing plib035_mflash.o(i.MFLASH_BusyStatus), (16 bytes).
    Removing plib035_mflash.o(i.MFLASH_EraseFull), (92 bytes).
    Removing plib035_mflash.o(i.MFLASH_ErasePage), (132 bytes).
    Removing plib035_mflash.o(i.MFLASH_ReadData), (212 bytes).
    Removing plib035_mflash.o(i.MFLASH_SetCmd), (20 bytes).
    Removing plib035_mflash.o(i.MFLASH_WriteData), (180 bytes).
    Removing plib035_pmu.o(.rev16_text), (4 bytes).
    Removing plib035_pmu.o(.revsh_text), (4 bytes).
    Removing plib035_pmu.o(.rrx_text), (6 bytes).
    Removing plib035_pwm.o(.rev16_text), (4 bytes).
    Removing plib035_pwm.o(.revsh_text), (4 bytes).
    Removing plib035_pwm.o(.rrx_text), (6 bytes).
    Removing plib035_pwm.o(i.PWM_AQ_ActionAConfig), (160 bytes).
    Removing plib035_pwm.o(i.PWM_AQ_ActionBConfig), (160 bytes).
    Removing plib035_pwm.o(i.PWM_AQ_Init), (130 bytes).
    Removing plib035_pwm.o(i.PWM_AQ_StructInit), (28 bytes).
    Removing plib035_pwm.o(i.PWM_CMP_CmpADirectLoadCmd), (112 bytes).
    Removing plib035_pwm.o(i.PWM_CMP_CmpALoadEventConfig), (120 bytes).
    Removing plib035_pwm.o(i.PWM_CMP_Init), (168 bytes).
    Removing plib035_pwm.o(i.PWM_CMP_StructInit), (16 bytes).
    Removing plib035_pwm.o(i.PWM_DB_Init), (292 bytes).
    Removing plib035_pwm.o(i.PWM_DB_StructInit), (14 bytes).
    Removing plib035_pwm.o(i.PWM_DeInit), (116 bytes).
    Removing plib035_pwm.o(i.PWM_ET_Init), (680 bytes).
    Removing plib035_pwm.o(i.PWM_ET_StructInit), (30 bytes).
    Removing plib035_pwm.o(i.PWM_HD_Init), (336 bytes).
    Removing plib035_pwm.o(i.PWM_HD_StructInit), (16 bytes).
    Removing plib035_pwm.o(i.PWM_TB_ClkDivConfig), (152 bytes).
    Removing plib035_pwm.o(i.PWM_TB_Init), (532 bytes).
    Removing plib035_pwm.o(i.PWM_TB_StructInit), (24 bytes).
    Removing plib035_pwm.o(i.PWM_TZ_Init), (248 bytes).
    Removing plib035_pwm.o(i.PWM_TZ_StructInit), (12 bytes).
    Removing plib035_pwm.o(i.RCU_APBRstCmd), (152 bytes).
    Removing plib035_qep.o(.rev16_text), (4 bytes).
    Removing plib035_qep.o(.revsh_text), (4 bytes).
    Removing plib035_qep.o(.rrx_text), (6 bytes).
    Removing plib035_qep.o(i.QEP_CAP_Init), (224 bytes).
    Removing plib035_qep.o(i.QEP_CAP_StructInit), (18 bytes).
    Removing plib035_qep.o(i.QEP_CMP_Init), (180 bytes).
    Removing plib035_qep.o(i.QEP_CMP_StructInit), (18 bytes).
    Removing plib035_qep.o(i.QEP_DeInit), (26 bytes).
    Removing plib035_qep.o(i.QEP_PC_Init), (280 bytes).
    Removing plib035_qep.o(i.QEP_PC_StructInit), (24 bytes).
    Removing plib035_qep.o(i.RCU_APBRstCmd), (152 bytes).
    Removing plib035_rcu.o(.rev16_text), (4 bytes).
    Removing plib035_rcu.o(.revsh_text), (4 bytes).
    Removing plib035_rcu.o(.rrx_text), (6 bytes).
    Removing plib035_rcu.o(i.RCU_GetADCClkFreq), (48 bytes).
    Removing plib035_rcu.o(i.RCU_GetClkOutFreq), (44 bytes).
    Removing plib035_rcu.o(i.RCU_GetOSEClkFreq), (8 bytes).
    Removing plib035_rcu.o(i.RCU_GetOSIClkFreq), (8 bytes).
    Removing plib035_rcu.o(i.RCU_GetPLLClkFreq), (56 bytes).
    Removing plib035_rcu.o(i.RCU_GetPLLDivClkFreq), (28 bytes).
    Removing plib035_rcu.o(i.RCU_GetSPIClkFreq), (48 bytes).
    Removing plib035_rcu.o(i.RCU_GetSysClkFreq), (16 bytes).
    Removing plib035_rcu.o(i.RCU_GetTraceClkFreq), (44 bytes).
    Removing plib035_rcu.o(i.RCU_GetUARTClkFreq), (48 bytes).
    Removing plib035_rcu.o(i.RCU_GetWDTClkFreq), (44 bytes).
    Removing plib035_rcu.o(i.RCU_PLL_DeInit), (24 bytes).
    Removing plib035_rcu.o(i.getPeriphClkFreq), (38 bytes).
    Removing plib035_rcu.o(i.getSysClkFreq), (38 bytes).
    Removing plib035_rcu.o(i.getSysPeriphClkFreq), (38 bytes).
    Removing plib035_spi.o(.rev16_text), (4 bytes).
    Removing plib035_spi.o(.revsh_text), (4 bytes).
    Removing plib035_spi.o(.rrx_text), (6 bytes).
    Removing plib035_spi.o(i.RCU_SPIRstCmd), (80 bytes).
    Removing plib035_spi.o(i.SPI_DeInit), (18 bytes).
    Removing plib035_spi.o(i.SPI_Init), (228 bytes).
    Removing plib035_spi.o(i.SPI_StructInit), (18 bytes).
    Removing plib035_tmr.o(.rev16_text), (4 bytes).
    Removing plib035_tmr.o(.revsh_text), (4 bytes).
    Removing plib035_tmr.o(.rrx_text), (6 bytes).
    Removing plib035_tmr.o(i.TMR_FreqConfig), (8 bytes).
    Removing plib035_tmr.o(i.TMR_PeriodConfig), (16 bytes).
    Removing plib035_tmr.o(i.TMR_SetLoad), (100 bytes).
    Removing plib035_uart.o(.rev16_text), (4 bytes).
    Removing plib035_uart.o(.revsh_text), (4 bytes).
    Removing plib035_uart.o(.rrx_text), (6 bytes).
    Removing plib035_uart.o(i.RCU_UARTRstCmd), (84 bytes).
    Removing plib035_uart.o(i.UART_AutoBaudConfig), (260 bytes).
    Removing plib035_uart.o(i.UART_DeInit), (100 bytes).
    Removing plib035_uart.o(i.UART_Init), (316 bytes).
    Removing plib035_uart.o(i.UART_StructInit), (24 bytes).
    Removing plib035_wdt.o(.rev16_text), (4 bytes).
    Removing plib035_wdt.o(.revsh_text), (4 bytes).
    Removing plib035_wdt.o(.rrx_text), (6 bytes).
    Removing retarget.o(.rev16_text), (4 bytes).
    Removing retarget.o(.revsh_text), (4 bytes).
    Removing retarget.o(.rrx_text), (6 bytes).
    Removing retarget.o(i._ttywrch), (4 bytes).
    Removing retarget.o(i.fgetc), (4 bytes).
    Removing retarget.o(.data), (4 bytes).
    Removing retarget_conf.o(.rev16_text), (4 bytes).
    Removing retarget_conf.o(.revsh_text), (4 bytes).
    Removing retarget_conf.o(.rrx_text), (6 bytes).
    Removing retarget_conf.o(i.retarget_get_char), (20 bytes).

159 unused section(s) (total 11136 bytes) removed from the image.

==============================================================================

Image Symbol Table

    Local Symbols

    Symbol Name                              Value     Ov Type        Size  Object(Section)

    RESET                                    0x00000000   Section      344  startup_k1921vk035.o(RESET)
    ../clib/angel/boardlib.s                 0x00000000   Number         0  boardshut.o ABSOLUTE
    ../clib/angel/boardlib.s                 0x00000000   Number         0  boardinit3.o ABSOLUTE
    ../clib/angel/boardlib.s                 0x00000000   Number         0  boardinit2.o ABSOLUTE
    ../clib/angel/boardlib.s                 0x00000000   Number         0  boardinit1.o ABSOLUTE
    ../clib/angel/dczerorl2.s                0x00000000   Number         0  __dczerorl2.o ABSOLUTE
    ../clib/angel/handlers.s                 0x00000000   Number         0  __scatter_zi.o ABSOLUTE
    ../clib/angel/kernel.s                   0x00000000   Number         0  __rtentry.o ABSOLUTE
    ../clib/angel/kernel.s                   0x00000000   Number         0  rtexit2.o ABSOLUTE
    ../clib/angel/kernel.s                   0x00000000   Number         0  __rtentry2.o ABSOLUTE
    ../clib/angel/kernel.s                   0x00000000   Number         0  rtexit.o ABSOLUTE
    ../clib/angel/kernel.s                   0x00000000   Number         0  __rtentry4.o ABSOLUTE
    ../clib/angel/rt.s                       0x00000000   Number         0  rt_raise.o ABSOLUTE
    ../clib/angel/scatter.s                  0x00000000   Number         0  __scatter.o ABSOLUTE
    ../clib/angel/startup.s                  0x00000000   Number         0  __main.o ABSOLUTE
    ../clib/angel/sys.s                      0x00000000   Number         0  sys_stackheap_outer.o ABSOLUTE
    ../clib/angel/sys.s                      0x00000000   Number         0  indicate_semi.o ABSOLUTE
    ../clib/angel/sys.s                      0x00000000   Number         0  use_no_semi.o ABSOLUTE
    ../clib/angel/sys.s                      0x00000000   Number         0  libspace.o ABSOLUTE
    ../clib/angel/sysapp.c                   0x00000000   Number         0  sys_command.o ABSOLUTE
    ../clib/armsys.c                         0x00000000   Number         0  argv_veneer.o ABSOLUTE
    ../clib/armsys.c                         0x00000000   Number         0  argv_veneer.o ABSOLUTE
    ../clib/armsys.c                         0x00000000   Number         0  _get_argv_nomalloc.o ABSOLUTE
    ../clib/armsys.c                         0x00000000   Number         0  no_argv.o ABSOLUTE
    ../clib/heapalloc.c                      0x00000000   Number         0  hrguard.o ABSOLUTE
    ../clib/heapaux.c                        0x00000000   Number         0  heapauxi.o ABSOLUTE
    ../clib/libinit.s                        0x00000000   Number         0  libshutdown.o ABSOLUTE
    ../clib/libinit.s                        0x00000000   Number         0  libshutdown2.o ABSOLUTE
    ../clib/libinit.s                        0x00000000   Number         0  libinit2.o ABSOLUTE
    ../clib/libinit.s                        0x00000000   Number         0  libinit.o ABSOLUTE
    ../clib/misc.s                           0x00000000   Number         0  printf_stubs.o ABSOLUTE
    ../clib/printf.c                         0x00000000   Number         0  _printf_dec.o ABSOLUTE
    ../clib/printf.c                         0x00000000   Number         0  __printf_ss.o ABSOLUTE
    ../clib/printf.c                         0x00000000   Number         0  __printf_flags_ss.o ABSOLUTE
    ../clib/printf.c                         0x00000000   Number         0  __printf_wp.o ABSOLUTE
    ../clib/printf.c                         0x00000000   Number         0  __printf_flags_wp.o ABSOLUTE
    ../clib/printf.c                         0x00000000   Number         0  __printf_flags.o ABSOLUTE
    ../clib/printf.c                         0x00000000   Number         0  __printf_flags_ss_wp.o ABSOLUTE
    ../clib/printf.c                         0x00000000   Number         0  __printf_nopercent.o ABSOLUTE
    ../clib/printf.c                         0x00000000   Number         0  __printf_ss_wp.o ABSOLUTE
    ../clib/printf.c                         0x00000000   Number         0  _printf_char_file.o ABSOLUTE
    ../clib/printf.c                         0x00000000   Number         0  _printf_char.o ABSOLUTE
    ../clib/printf.c                         0x00000000   Number         0  _printf_intcommon.o ABSOLUTE
    ../clib/printf.c                         0x00000000   Number         0  _printf_char_common.o ABSOLUTE
    ../clib/printf.c                         0x00000000   Number         0  __2printf.o ABSOLUTE
    ../clib/printf.c                         0x00000000   Number         0  noretval__2printf.o ABSOLUTE
    ../clib/printf.c                         0x00000000   Number         0  __printf.o ABSOLUTE
    ../clib/printf.c                         0x00000000   Number         0  _printf_pad.o ABSOLUTE
    ../clib/printf.c                         0x00000000   Number         0  _printf_str.o ABSOLUTE
    ../clib/printf_percent.s                 0x00000000   Number         0  _printf_percent_end.o ABSOLUTE
    ../clib/printf_percent.s                 0x00000000   Number         0  _printf_s.o ABSOLUTE
    ../clib/printf_percent.s                 0x00000000   Number         0  _printf_d.o ABSOLUTE
    ../clib/printf_percent.s                 0x00000000   Number         0  _printf_percent.o ABSOLUTE
    ../clib/signal.c                         0x00000000   Number         0  defsig_rtred_inner.o ABSOLUTE
    ../clib/signal.c                         0x00000000   Number         0  defsig_stak_inner.o ABSOLUTE
    ../clib/signal.c                         0x00000000   Number         0  defsig_pvfn_inner.o ABSOLUTE
    ../clib/signal.c                         0x00000000   Number         0  defsig_cppl_inner.o ABSOLUTE
    ../clib/signal.c                         0x00000000   Number         0  defsig_segv_inner.o ABSOLUTE
    ../clib/signal.c                         0x00000000   Number         0  defsig_other.o ABSOLUTE
    ../clib/signal.c                         0x00000000   Number         0  defsig_rtmem_inner.o ABSOLUTE
    ../clib/signal.c                         0x00000000   Number         0  __raise.o ABSOLUTE
    ../clib/signal.c                         0x00000000   Number         0  defsig_rtmem_formal.o ABSOLUTE
    ../clib/signal.c                         0x00000000   Number         0  defsig_rtmem_outer.o ABSOLUTE
    ../clib/signal.c                         0x00000000   Number         0  defsig_general.o ABSOLUTE
    ../clib/signal.c                         0x00000000   Number         0  defsig_abrt_inner.o ABSOLUTE
    ../clib/signal.c                         0x00000000   Number         0  defsig_exit.o ABSOLUTE
    ../clib/signal.c                         0x00000000   Number         0  defsig_fpe_inner.o ABSOLUTE
    ../clib/signal.s                         0x00000000   Number         0  defsig.o ABSOLUTE
    ../clib/stdlib.c                         0x00000000   Number         0  exit.o ABSOLUTE
    ../fplib/ddiv.s                          0x00000000   Number         0  ddiv.o ABSOLUTE
    ../fplib/dfix.s                          0x00000000   Number         0  dfix.o ABSOLUTE
    ../fplib/dflt.s                          0x00000000   Number         0  dflt_clz.o ABSOLUTE
    ../fplib/dnaninf.s                       0x00000000   Number         0  dnaninf.o ABSOLUTE
    ../fplib/dretinf.s                       0x00000000   Number         0  dretinf.o ABSOLUTE
    ../fplib/fpinit.s                        0x00000000   Number         0  fpinit.o ABSOLUTE
    ../fplib/usenofp.s                       0x00000000   Number         0  usenofp.o ABSOLUTE
    Core\App\gpio.c                          0x00000000   Number         0  gpio.o ABSOLUTE
    Core\App\main.c                          0x00000000   Number         0  main.o ABSOLUTE
    Core\App\rcu.c                           0x00000000   Number         0  rcu.o ABSOLUTE
    Core\App\vk035_it.c                      0x00000000   Number         0  vk035_it.o ABSOLUTE
    Core\\App\\gpio.c                        0x00000000   Number         0  gpio.o ABSOLUTE
    Core\\App\\main.c                        0x00000000   Number         0  main.o ABSOLUTE
    Core\\App\\rcu.c                         0x00000000   Number         0  rcu.o ABSOLUTE
    Core\\App\\vk035_it.c                    0x00000000   Number         0  vk035_it.o ABSOLUTE
    dc.s                                     0x00000000   Number         0  dc.o ABSOLUTE
    platform\Device\NIIET\K1921VK035\Source\ARM\startup_K1921VK035.s 0x00000000   Number         0  startup_k1921vk035.o ABSOLUTE
    platform\Device\NIIET\K1921VK035\Source\system_K1921VK035.c 0x00000000   Number         0  system_k1921vk035.o ABSOLUTE
    platform\\Device\\NIIET\\K1921VK035\\Source\\system_K1921VK035.c 0x00000000   Number         0  system_k1921vk035.o ABSOLUTE
    platform\\plib035\\src\\plib035_adc.c    0x00000000   Number         0  plib035_adc.o ABSOLUTE
    platform\\plib035\\src\\plib035_can.c    0x00000000   Number         0  plib035_can.o ABSOLUTE
    platform\\plib035\\src\\plib035_dma.c    0x00000000   Number         0  plib035_dma.o ABSOLUTE
    platform\\plib035\\src\\plib035_ecap.c   0x00000000   Number         0  plib035_ecap.o ABSOLUTE
    platform\\plib035\\src\\plib035_gpio.c   0x00000000   Number         0  plib035_gpio.o ABSOLUTE
    platform\\plib035\\src\\plib035_i2c.c    0x00000000   Number         0  plib035_i2c.o ABSOLUTE
    platform\\plib035\\src\\plib035_mflash.c 0x00000000   Number         0  plib035_mflash.o ABSOLUTE
    platform\\plib035\\src\\plib035_pmu.c    0x00000000   Number         0  plib035_pmu.o ABSOLUTE
    platform\\plib035\\src\\plib035_pwm.c    0x00000000   Number         0  plib035_pwm.o ABSOLUTE
    platform\\plib035\\src\\plib035_qep.c    0x00000000   Number         0  plib035_qep.o ABSOLUTE
    platform\\plib035\\src\\plib035_rcu.c    0x00000000   Number         0  plib035_rcu.o ABSOLUTE
    platform\\plib035\\src\\plib035_spi.c    0x00000000   Number         0  plib035_spi.o ABSOLUTE
    platform\\plib035\\src\\plib035_tmr.c    0x00000000   Number         0  plib035_tmr.o ABSOLUTE
    platform\\plib035\\src\\plib035_uart.c   0x00000000   Number         0  plib035_uart.o ABSOLUTE
    platform\\plib035\\src\\plib035_wdt.c    0x00000000   Number         0  plib035_wdt.o ABSOLUTE
    platform\\retarget\\retarget.c           0x00000000   Number         0  retarget.o ABSOLUTE
    platform\\retarget\\retarget_conf.c      0x00000000   Number         0  retarget_conf.o ABSOLUTE
    platform\plib035\src\plib035_adc.c       0x00000000   Number         0  plib035_adc.o ABSOLUTE
    platform\plib035\src\plib035_can.c       0x00000000   Number         0  plib035_can.o ABSOLUTE
    platform\plib035\src\plib035_dma.c       0x00000000   Number         0  plib035_dma.o ABSOLUTE
    platform\plib035\src\plib035_ecap.c      0x00000000   Number         0  plib035_ecap.o ABSOLUTE
    platform\plib035\src\plib035_gpio.c      0x00000000   Number         0  plib035_gpio.o ABSOLUTE
    platform\plib035\src\plib035_i2c.c       0x00000000   Number         0  plib035_i2c.o ABSOLUTE
    platform\plib035\src\plib035_mflash.c    0x00000000   Number         0  plib035_mflash.o ABSOLUTE
    platform\plib035\src\plib035_pmu.c       0x00000000   Number         0  plib035_pmu.o ABSOLUTE
    platform\plib035\src\plib035_pwm.c       0x00000000   Number         0  plib035_pwm.o ABSOLUTE
    platform\plib035\src\plib035_qep.c       0x00000000   Number         0  plib035_qep.o ABSOLUTE
    platform\plib035\src\plib035_rcu.c       0x00000000   Number         0  plib035_rcu.o ABSOLUTE
    platform\plib035\src\plib035_spi.c       0x00000000   Number         0  plib035_spi.o ABSOLUTE
    platform\plib035\src\plib035_tmr.c       0x00000000   Number         0  plib035_tmr.o ABSOLUTE
    platform\plib035\src\plib035_uart.c      0x00000000   Number         0  plib035_uart.o ABSOLUTE
    platform\plib035\src\plib035_wdt.c       0x00000000   Number         0  plib035_wdt.o ABSOLUTE
    platform\retarget\retarget.c             0x00000000   Number         0  retarget.o ABSOLUTE
    platform\retarget\retarget_conf.c        0x00000000   Number         0  retarget_conf.o ABSOLUTE
    !!!main                                  0x00000158   Section        8  __main.o(!!!main)
    !!!scatter                               0x00000160   Section       52  __scatter.o(!!!scatter)
    !!dczerorl2                              0x00000194   Section       90  __dczerorl2.o(!!dczerorl2)
    !!handler_zi                             0x000001f0   Section       28  __scatter_zi.o(!!handler_zi)
    .ARM.Collect$$_printf_percent$$00000000  0x0000020c   Section        0  _printf_percent.o(.ARM.Collect$$_printf_percent$$00000000)
    .ARM.Collect$$_printf_percent$$00000009  0x0000020c   Section        6  _printf_d.o(.ARM.Collect$$_printf_percent$$00000009)
    .ARM.Collect$$_printf_percent$$00000014  0x00000212   Section        6  _printf_s.o(.ARM.Collect$$_printf_percent$$00000014)
    .ARM.Collect$$_printf_percent$$00000017  0x00000218   Section        4  _printf_percent_end.o(.ARM.Collect$$_printf_percent$$00000017)
    .ARM.Collect$$libinit$$00000000          0x0000021c   Section        2  libinit.o(.ARM.Collect$$libinit$$00000000)
    .ARM.Collect$$libinit$$00000001          0x0000021e   Section        4  libinit2.o(.ARM.Collect$$libinit$$00000001)
    .ARM.Collect$$libinit$$00000004          0x00000222   Section        0  libinit2.o(.ARM.Collect$$libinit$$00000004)
    .ARM.Collect$$libinit$$0000000A          0x00000222   Section        0  libinit2.o(.ARM.Collect$$libinit$$0000000A)
    .ARM.Collect$$libinit$$0000000C          0x00000222   Section        0  libinit2.o(.ARM.Collect$$libinit$$0000000C)
    .ARM.Collect$$libinit$$0000000E          0x00000222   Section        0  libinit2.o(.ARM.Collect$$libinit$$0000000E)
    .ARM.Collect$$libinit$$00000011          0x00000222   Section        0  libinit2.o(.ARM.Collect$$libinit$$00000011)
    .ARM.Collect$$libinit$$00000013          0x00000222   Section        0  libinit2.o(.ARM.Collect$$libinit$$00000013)
    .ARM.Collect$$libinit$$00000015          0x00000222   Section        0  libinit2.o(.ARM.Collect$$libinit$$00000015)
    .ARM.Collect$$libinit$$00000017          0x00000222   Section        0  libinit2.o(.ARM.Collect$$libinit$$00000017)
    .ARM.Collect$$libinit$$00000019          0x00000222   Section        0  libinit2.o(.ARM.Collect$$libinit$$00000019)
    .ARM.Collect$$libinit$$0000001B          0x00000222   Section        0  libinit2.o(.ARM.Collect$$libinit$$0000001B)
    .ARM.Collect$$libinit$$0000001D          0x00000222   Section        0  libinit2.o(.ARM.Collect$$libinit$$0000001D)
    .ARM.Collect$$libinit$$0000001F          0x00000222   Section        0  libinit2.o(.ARM.Collect$$libinit$$0000001F)
    .ARM.Collect$$libinit$$00000021          0x00000222   Section        0  libinit2.o(.ARM.Collect$$libinit$$00000021)
    .ARM.Collect$$libinit$$00000023          0x00000222   Section        0  libinit2.o(.ARM.Collect$$libinit$$00000023)
    .ARM.Collect$$libinit$$00000025          0x00000222   Section        0  libinit2.o(.ARM.Collect$$libinit$$00000025)
    .ARM.Collect$$libinit$$0000002C          0x00000222   Section        0  libinit2.o(.ARM.Collect$$libinit$$0000002C)
    .ARM.Collect$$libinit$$0000002E          0x00000222   Section        0  libinit2.o(.ARM.Collect$$libinit$$0000002E)
    .ARM.Collect$$libinit$$00000030          0x00000222   Section        0  libinit2.o(.ARM.Collect$$libinit$$00000030)
    .ARM.Collect$$libinit$$00000032          0x00000222   Section        0  libinit2.o(.ARM.Collect$$libinit$$00000032)
    .ARM.Collect$$libinit$$00000033          0x00000222   Section        2  libinit2.o(.ARM.Collect$$libinit$$00000033)
    .ARM.Collect$$libshutdown$$00000000      0x00000224   Section        2  libshutdown.o(.ARM.Collect$$libshutdown$$00000000)
    .ARM.Collect$$libshutdown$$00000002      0x00000226   Section        0  libshutdown2.o(.ARM.Collect$$libshutdown$$00000002)
    .ARM.Collect$$libshutdown$$00000004      0x00000226   Section        0  libshutdown2.o(.ARM.Collect$$libshutdown$$00000004)
    .ARM.Collect$$libshutdown$$00000006      0x00000226   Section        0  libshutdown2.o(.ARM.Collect$$libshutdown$$00000006)
    .ARM.Collect$$libshutdown$$00000009      0x00000226   Section        0  libshutdown2.o(.ARM.Collect$$libshutdown$$00000009)
    .ARM.Collect$$libshutdown$$0000000C      0x00000226   Section        0  libshutdown2.o(.ARM.Collect$$libshutdown$$0000000C)
    .ARM.Collect$$libshutdown$$0000000E      0x00000226   Section        0  libshutdown2.o(.ARM.Collect$$libshutdown$$0000000E)
    .ARM.Collect$$libshutdown$$00000011      0x00000226   Section        0  libshutdown2.o(.ARM.Collect$$libshutdown$$00000011)
    .ARM.Collect$$libshutdown$$00000012      0x00000226   Section        2  libshutdown2.o(.ARM.Collect$$libshutdown$$00000012)
    .ARM.Collect$$rtentry$$00000000          0x00000228   Section        0  __rtentry.o(.ARM.Collect$$rtentry$$00000000)
    .ARM.Collect$$rtentry$$00000002          0x00000228   Section        0  __rtentry2.o(.ARM.Collect$$rtentry$$00000002)
    .ARM.Collect$$rtentry$$00000004          0x00000228   Section        6  __rtentry4.o(.ARM.Collect$$rtentry$$00000004)
    .ARM.Collect$$rtentry$$00000009          0x0000022e   Section        0  __rtentry2.o(.ARM.Collect$$rtentry$$00000009)
    .ARM.Collect$$rtentry$$0000000A          0x0000022e   Section        4  __rtentry2.o(.ARM.Collect$$rtentry$$0000000A)
    .ARM.Collect$$rtentry$$0000000C          0x00000232   Section        0  __rtentry2.o(.ARM.Collect$$rtentry$$0000000C)
    .ARM.Collect$$rtentry$$0000000D          0x00000232   Section        8  __rtentry2.o(.ARM.Collect$$rtentry$$0000000D)
    .ARM.Collect$$rtexit$$00000000           0x0000023a   Section        2  rtexit.o(.ARM.Collect$$rtexit$$00000000)
    .ARM.Collect$$rtexit$$00000002           0x0000023c   Section        0  rtexit2.o(.ARM.Collect$$rtexit$$00000002)
    .ARM.Collect$$rtexit$$00000003           0x0000023c   Section        4  rtexit2.o(.ARM.Collect$$rtexit$$00000003)
    .ARM.Collect$$rtexit$$00000004           0x00000240   Section        6  rtexit2.o(.ARM.Collect$$rtexit$$00000004)
    .text                                    0x00000248   Section       64  startup_k1921vk035.o(.text)
    $v0                                      0x00000248   Number         0  startup_k1921vk035.o(.text)
    .text                                    0x00000288   Section        2  use_no_semi.o(.text)
    .text                                    0x0000028c   Section        0  noretval__2printf.o(.text)
    .text                                    0x000002a4   Section        0  _printf_pad.o(.text)
    .text                                    0x000002f2   Section        0  _printf_str.o(.text)
    .text                                    0x00000344   Section        0  _printf_dec.o(.text)
    .text                                    0x000003bc   Section        0  __printf_wp.o(.text)
    .text                                    0x000004ca   Section        0  heapauxi.o(.text)
    .text                                    0x000004d0   Section        0  _printf_intcommon.o(.text)
    .text                                    0x00000582   Section        0  _printf_char.o(.text)
    .text                                    0x000005b0   Section        0  _printf_char_file.o(.text)
    .text                                    0x000005d4   Section        0  _printf_char_common.o(.text)
    _printf_input_char                       0x000005d5   Thumb Code    10  _printf_char_common.o(.text)
    .text                                    0x00000604   Section       74  sys_stackheap_outer.o(.text)
    .text                                    0x0000064e   Section        0  exit.o(.text)
    .text                                    0x00000660   Section        8  libspace.o(.text)
    i.BusFault_Handler                       0x00000668   Section        0  vk035_it.o(i.BusFault_Handler)
    i.ClkInit                                0x0000066c   Section        0  system_k1921vk035.o(i.ClkInit)
    i.DebugMon_Handler                       0x000006e0   Section        0  vk035_it.o(i.DebugMon_Handler)
    i.Error_Handler                          0x000006e2   Section        0  main.o(i.Error_Handler)
    i.FPUInit                                0x000006e8   Section        0  system_k1921vk035.o(i.FPUInit)
    i.GPIO_AltFuncCmd                        0x00000700   Section        0  plib035_gpio.o(i.GPIO_AltFuncCmd)
    GPIO_AltFuncCmd                          0x00000701   Thumb Code    74  plib035_gpio.o(i.GPIO_AltFuncCmd)
    i.GPIO_DeInit                            0x00000758   Section        0  plib035_gpio.o(i.GPIO_DeInit)
    i.GPIO_DigitalCmd                        0x000007bc   Section        0  plib035_gpio.o(i.GPIO_DigitalCmd)
    GPIO_DigitalCmd                          0x000007bd   Thumb Code    74  plib035_gpio.o(i.GPIO_DigitalCmd)
    i.GPIO_DriveModeConfig                   0x00000838   Section        0  plib035_gpio.o(i.GPIO_DriveModeConfig)
    i.GPIO_InModeConfig                      0x000008b4   Section        0  plib035_gpio.o(i.GPIO_InModeConfig)
    i.GPIO_Init                              0x0000092c   Section        0  plib035_gpio.o(i.GPIO_Init)
    i.GPIO_ModeConfig                        0x0000097c   Section        0  plib035_gpio.o(i.GPIO_ModeConfig)
    GPIO_ModeConfig                          0x0000097d   Thumb Code    44  plib035_gpio.o(i.GPIO_ModeConfig)
    i.GPIO_OutCmd                            0x000009a8   Section        0  plib035_gpio.o(i.GPIO_OutCmd)
    GPIO_OutCmd                              0x000009a9   Thumb Code    74  plib035_gpio.o(i.GPIO_OutCmd)
    i.GPIO_OutModeConfig                     0x00000a00   Section        0  plib035_gpio.o(i.GPIO_OutModeConfig)
    i.GPIO_PullModeConfig                    0x00000a78   Section        0  plib035_gpio.o(i.GPIO_PullModeConfig)
    i.HardFault_Handler                      0x00000af0   Section        0  vk035_it.o(i.HardFault_Handler)
    i.MFLASH_LatencyConfig                   0x00000af4   Section        0  plib035_rcu.o(i.MFLASH_LatencyConfig)
    MFLASH_LatencyConfig                     0x00000af5   Thumb Code    28  plib035_rcu.o(i.MFLASH_LatencyConfig)
    i.MemManage_Handler                      0x00000b3c   Section        0  vk035_it.o(i.MemManage_Handler)
    i.NMI_Handler                            0x00000b3e   Section        0  vk035_it.o(i.NMI_Handler)
    i.PendSV_Handler                         0x00000b40   Section        0  vk035_it.o(i.PendSV_Handler)
    i.RCU_AHBRstCmd                          0x00000b44   Section        0  plib035_gpio.o(i.RCU_AHBRstCmd)
    RCU_AHBRstCmd                            0x00000b45   Thumb Code    64  plib035_gpio.o(i.RCU_AHBRstCmd)
    i.RCU_ClkOutConfig                       0x00000bb0   Section        0  rcu.o(i.RCU_ClkOutConfig)
    RCU_ClkOutConfig                         0x00000bb1   Thumb Code    86  rcu.o(i.RCU_ClkOutConfig)
    i.RCU_PLL_AutoConfig                     0x00000c38   Section        0  plib035_rcu.o(i.RCU_PLL_AutoConfig)
    i.RCU_PLL_Init                           0x00000d98   Section        0  plib035_rcu.o(i.RCU_PLL_Init)
    i.RCU_PLL_OutCmd                         0x00000e98   Section        0  plib035_rcu.o(i.RCU_PLL_OutCmd)
    RCU_PLL_OutCmd                           0x00000e99   Thumb Code    34  plib035_rcu.o(i.RCU_PLL_OutCmd)
    i.RCU_PLL_StructInit                     0x00000ee8   Section        0  plib035_rcu.o(i.RCU_PLL_StructInit)
    i.RCU_SysClkChangeCmd                    0x00000ef8   Section        0  plib035_rcu.o(i.RCU_SysClkChangeCmd)
    i.SVC_Handler                            0x00000fb0   Section        0  vk035_it.o(i.SVC_Handler)
    i.SysTick_Handler                        0x00000fb4   Section        0  vk035_it.o(i.SysTick_Handler)
    i.SystemCoreClockUpdate                  0x00000fc4   Section        0  system_k1921vk035.o(i.SystemCoreClockUpdate)
    i.SystemInit                             0x00001034   Section        0  system_k1921vk035.o(i.SystemInit)
    i.UsageFault_Handler                     0x00001042   Section        0  vk035_it.o(i.UsageFault_Handler)
    i._is_digit                              0x00001044   Section        0  __printf_wp.o(i._is_digit)
    i._sys_exit                              0x00001052   Section        0  retarget.o(i._sys_exit)
    i.assert_failed                          0x00001054   Section        0  main.o(i.assert_failed)
    i.ferror                                 0x00001084   Section        0  retarget.o(i.ferror)
    i.fputc                                  0x0000108a   Section        0  retarget.o(i.fputc)
    i.gpio_init                              0x00001090   Section        0  gpio.o(i.gpio_init)
    i.main                                   0x00001104   Section        0  main.o(i.main)
    i.periph_init                            0x0000110c   Section        0  main.o(i.periph_init)
    i.retarget_init                          0x0000117c   Section        0  retarget_conf.o(i.retarget_init)
    i.retarget_put_char                      0x0000123c   Section        0  retarget_conf.o(i.retarget_put_char)
    i.sysclk_init                            0x00001250   Section        0  rcu.o(i.sysclk_init)
    x$fpl$ddiv                               0x000012b8   Section      688  ddiv.o(x$fpl$ddiv)
    $v0                                      0x000012b8   Number         0  ddiv.o(x$fpl$ddiv)
    ddiv_entry                               0x000012bf   Thumb Code     0  ddiv.o(x$fpl$ddiv)
    x$fpl$dfix                               0x00001568   Section       94  dfix.o(x$fpl$dfix)
    $v0                                      0x00001568   Number         0  dfix.o(x$fpl$dfix)
    x$fpl$dfltu                              0x000015c6   Section       38  dflt_clz.o(x$fpl$dfltu)
    $v0                                      0x000015c6   Number         0  dflt_clz.o(x$fpl$dfltu)
    x$fpl$dnaninf                            0x000015ec   Section      156  dnaninf.o(x$fpl$dnaninf)
    $v0                                      0x000015ec   Number         0  dnaninf.o(x$fpl$dnaninf)
    x$fpl$dretinf                            0x00001688   Section       12  dretinf.o(x$fpl$dretinf)
    $v0                                      0x00001688   Number         0  dretinf.o(x$fpl$dretinf)
    x$fpl$fpinit                             0x00001694   Section       10  fpinit.o(x$fpl$fpinit)
    $v0                                      0x00001694   Number         0  fpinit.o(x$fpl$fpinit)
    x$fpl$usenofp                            0x0000169e   Section        0  usenofp.o(x$fpl$usenofp)
    .data                                    0x20000000   Section        4  system_k1921vk035.o(.data)
    .data                                    0x20000004   Section        4  system_k1921vk035.o(.data)
    .data                                    0x20000008   Section      384  gpio.o(.data)
    gpioa_config                             0x20000008   Data         192  gpio.o(.data)
    gpiob_config                             0x200000c8   Data         192  gpio.o(.data)
    .data                                    0x20000188   Section        1  rcu.o(.data)
    OS_Type                                  0x20000188   Data           1  rcu.o(.data)
    .data                                    0x2000018c   Section        4  retarget.o(.data)
    .bss                                     0x20000190   Section       96  libspace.o(.bss)
    HEAP                                     0x200001f0   Section      512  startup_k1921vk035.o(HEAP)
    Heap_Mem                                 0x200001f0   Data         512  startup_k1921vk035.o(HEAP)
    STACK                                    0x200003f0   Section     1024  startup_k1921vk035.o(STACK)
    Stack_Mem                                0x200003f0   Data        1024  startup_k1921vk035.o(STACK)
    __initial_sp                             0x200007f0   Data           0  startup_k1921vk035.o(STACK)

    Global Symbols

    Symbol Name                              Value     Ov Type        Size  Object(Section)

    BuildAttributes$$THM_ISAv4$E$P$D$K$B$S$7EM$VFPi3$EXTD16$VFPS$VFMA$PE$A:L22UL41UL21$X:L11$S22US41US21$IEEE1$IW$USESV6$~STKCKD$USESV7$~SHL$OSPACE$ROPI$EBA8$UX$STANDARDLIB$REQ8$PRES8$EABIv2 0x00000000   Number         0  anon$$obj.o ABSOLUTE
    __ARM_use_no_argv                        0x00000000   Number         0  main.o ABSOLUTE
    __Vectors                                0x00000000   Data           4  startup_k1921vk035.o(RESET)
    _printf_flags                            0x00000000   Number         0  printf_stubs.o ABSOLUTE
    _printf_return_value                     0x00000000   Number         0  printf_stubs.o ABSOLUTE
    _printf_sizespec                         0x00000000   Number         0  printf_stubs.o ABSOLUTE
    _printf_widthprec                        0x00000000   Number         0  printf_stubs.o ABSOLUTE
    __ARM_exceptions_init                     - Undefined Weak Reference
    __alloca_initialize                       - Undefined Weak Reference
    __arm_fini_                               - Undefined Weak Reference
    __arm_preinit_                            - Undefined Weak Reference
    __cpp_initialize__aeabi_                  - Undefined Weak Reference
    __cxa_finalize                            - Undefined Weak Reference
    __rt_locale                               - Undefined Weak Reference
    __sigvec_lookup                           - Undefined Weak Reference
    _atexit_init                              - Undefined Weak Reference
    _call_atexit_fns                          - Undefined Weak Reference
    _clock_init                               - Undefined Weak Reference
    _fp_trap_init                             - Undefined Weak Reference
    _fp_trap_shutdown                         - Undefined Weak Reference
    _get_lc_collate                           - Undefined Weak Reference
    _get_lc_ctype                             - Undefined Weak Reference
    _get_lc_monetary                          - Undefined Weak Reference
    _get_lc_numeric                           - Undefined Weak Reference
    _get_lc_time                              - Undefined Weak Reference
    _getenv_init                              - Undefined Weak Reference
    _handle_redirection                       - Undefined Weak Reference
    _init_alloc                               - Undefined Weak Reference
    _init_user_alloc                          - Undefined Weak Reference
    _initio                                   - Undefined Weak Reference
    _printf_mbtowc                            - Undefined Weak Reference
    _printf_truncate_signed                   - Undefined Weak Reference
    _printf_truncate_unsigned                 - Undefined Weak Reference
    _rand_init                                - Undefined Weak Reference
    _signal_finish                            - Undefined Weak Reference
    _signal_init                              - Undefined Weak Reference
    _terminate_alloc                          - Undefined Weak Reference
    _terminate_user_alloc                     - Undefined Weak Reference
    _terminateio                              - Undefined Weak Reference
    __Vectors_End                            0x00000158   Data           0  startup_k1921vk035.o(RESET)
    __Vectors_Size                           0x00000158   Number         0  startup_k1921vk035.o ABSOLUTE
    __main                                   0x00000159   Thumb Code     8  __main.o(!!!main)
    __scatterload                            0x00000161   Thumb Code     0  __scatter.o(!!!scatter)
    __scatterload_rt2                        0x00000161   Thumb Code    44  __scatter.o(!!!scatter)
    __scatterload_rt2_thumb_only             0x00000161   Thumb Code     0  __scatter.o(!!!scatter)
    __scatterload_null                       0x0000016f   Thumb Code     0  __scatter.o(!!!scatter)
    __decompress                             0x00000195   Thumb Code    90  __dczerorl2.o(!!dczerorl2)
    __decompress1                            0x00000195   Thumb Code     0  __dczerorl2.o(!!dczerorl2)
    __scatterload_zeroinit                   0x000001f1   Thumb Code    28  __scatter_zi.o(!!handler_zi)
    _printf_d                                0x0000020d   Thumb Code     0  _printf_d.o(.ARM.Collect$$_printf_percent$$00000009)
    _printf_percent                          0x0000020d   Thumb Code     0  _printf_percent.o(.ARM.Collect$$_printf_percent$$00000000)
    _printf_s                                0x00000213   Thumb Code     0  _printf_s.o(.ARM.Collect$$_printf_percent$$00000014)
    _printf_percent_end                      0x00000219   Thumb Code     0  _printf_percent_end.o(.ARM.Collect$$_printf_percent$$00000017)
    __rt_lib_init                            0x0000021d   Thumb Code     0  libinit.o(.ARM.Collect$$libinit$$00000000)
    __rt_lib_init_fp_1                       0x0000021f   Thumb Code     0  libinit2.o(.ARM.Collect$$libinit$$00000001)
    __rt_lib_init_alloca_1                   0x00000223   Thumb Code     0  libinit2.o(.ARM.Collect$$libinit$$0000002E)
    __rt_lib_init_argv_1                     0x00000223   Thumb Code     0  libinit2.o(.ARM.Collect$$libinit$$0000002C)
    __rt_lib_init_atexit_1                   0x00000223   Thumb Code     0  libinit2.o(.ARM.Collect$$libinit$$0000001B)
    __rt_lib_init_clock_1                    0x00000223   Thumb Code     0  libinit2.o(.ARM.Collect$$libinit$$00000021)
    __rt_lib_init_cpp_1                      0x00000223   Thumb Code     0  libinit2.o(.ARM.Collect$$libinit$$00000032)
    __rt_lib_init_exceptions_1               0x00000223   Thumb Code     0  libinit2.o(.ARM.Collect$$libinit$$00000030)
    __rt_lib_init_fp_trap_1                  0x00000223   Thumb Code     0  libinit2.o(.ARM.Collect$$libinit$$0000001F)
    __rt_lib_init_getenv_1                   0x00000223   Thumb Code     0  libinit2.o(.ARM.Collect$$libinit$$00000023)
    __rt_lib_init_heap_1                     0x00000223   Thumb Code     0  libinit2.o(.ARM.Collect$$libinit$$0000000A)
    __rt_lib_init_lc_collate_1               0x00000223   Thumb Code     0  libinit2.o(.ARM.Collect$$libinit$$00000011)
    __rt_lib_init_lc_ctype_1                 0x00000223   Thumb Code     0  libinit2.o(.ARM.Collect$$libinit$$00000013)
    __rt_lib_init_lc_monetary_1              0x00000223   Thumb Code     0  libinit2.o(.ARM.Collect$$libinit$$00000015)
    __rt_lib_init_lc_numeric_1               0x00000223   Thumb Code     0  libinit2.o(.ARM.Collect$$libinit$$00000017)
    __rt_lib_init_lc_time_1                  0x00000223   Thumb Code     0  libinit2.o(.ARM.Collect$$libinit$$00000019)
    __rt_lib_init_preinit_1                  0x00000223   Thumb Code     0  libinit2.o(.ARM.Collect$$libinit$$00000004)
    __rt_lib_init_rand_1                     0x00000223   Thumb Code     0  libinit2.o(.ARM.Collect$$libinit$$0000000E)
    __rt_lib_init_return                     0x00000223   Thumb Code     0  libinit2.o(.ARM.Collect$$libinit$$00000033)
    __rt_lib_init_signal_1                   0x00000223   Thumb Code     0  libinit2.o(.ARM.Collect$$libinit$$0000001D)
    __rt_lib_init_stdio_1                    0x00000223   Thumb Code     0  libinit2.o(.ARM.Collect$$libinit$$00000025)
    __rt_lib_init_user_alloc_1               0x00000223   Thumb Code     0  libinit2.o(.ARM.Collect$$libinit$$0000000C)
    __rt_lib_shutdown                        0x00000225   Thumb Code     0  libshutdown.o(.ARM.Collect$$libshutdown$$00000000)
    __rt_lib_shutdown_cpp_1                  0x00000227   Thumb Code     0  libshutdown2.o(.ARM.Collect$$libshutdown$$00000004)
    __rt_lib_shutdown_fini_1                 0x00000227   Thumb Code     0  libshutdown2.o(.ARM.Collect$$libshutdown$$00000002)
    __rt_lib_shutdown_fp_trap_1              0x00000227   Thumb Code     0  libshutdown2.o(.ARM.Collect$$libshutdown$$00000009)
    __rt_lib_shutdown_heap_1                 0x00000227   Thumb Code     0  libshutdown2.o(.ARM.Collect$$libshutdown$$00000011)
    __rt_lib_shutdown_return                 0x00000227   Thumb Code     0  libshutdown2.o(.ARM.Collect$$libshutdown$$00000012)
    __rt_lib_shutdown_signal_1               0x00000227   Thumb Code     0  libshutdown2.o(.ARM.Collect$$libshutdown$$0000000C)
    __rt_lib_shutdown_stdio_1                0x00000227   Thumb Code     0  libshutdown2.o(.ARM.Collect$$libshutdown$$00000006)
    __rt_lib_shutdown_user_alloc_1           0x00000227   Thumb Code     0  libshutdown2.o(.ARM.Collect$$libshutdown$$0000000E)
    __rt_entry                               0x00000229   Thumb Code     0  __rtentry.o(.ARM.Collect$$rtentry$$00000000)
    __rt_entry_presh_1                       0x00000229   Thumb Code     0  __rtentry2.o(.ARM.Collect$$rtentry$$00000002)
    __rt_entry_sh                            0x00000229   Thumb Code     0  __rtentry4.o(.ARM.Collect$$rtentry$$00000004)
    __rt_entry_li                            0x0000022f   Thumb Code     0  __rtentry2.o(.ARM.Collect$$rtentry$$0000000A)
    __rt_entry_postsh_1                      0x0000022f   Thumb Code     0  __rtentry2.o(.ARM.Collect$$rtentry$$00000009)
    __rt_entry_main                          0x00000233   Thumb Code     0  __rtentry2.o(.ARM.Collect$$rtentry$$0000000D)
    __rt_entry_postli_1                      0x00000233   Thumb Code     0  __rtentry2.o(.ARM.Collect$$rtentry$$0000000C)
    __rt_exit                                0x0000023b   Thumb Code     0  rtexit.o(.ARM.Collect$$rtexit$$00000000)
    __rt_exit_ls                             0x0000023d   Thumb Code     0  rtexit2.o(.ARM.Collect$$rtexit$$00000003)
    __rt_exit_prels_1                        0x0000023d   Thumb Code     0  rtexit2.o(.ARM.Collect$$rtexit$$00000002)
    __rt_exit_exit                           0x00000241   Thumb Code     0  rtexit2.o(.ARM.Collect$$rtexit$$00000004)
    Reset_Handler                            0x00000249   Thumb Code     8  startup_k1921vk035.o(.text)
    ADC_DC_IRQHandler                        0x00000263   Thumb Code     0  startup_k1921vk035.o(.text)
    ADC_SEQ0_IRQHandler                      0x00000263   Thumb Code     0  startup_k1921vk035.o(.text)
    ADC_SEQ1_IRQHandler                      0x00000263   Thumb Code     0  startup_k1921vk035.o(.text)
    CAN0_IRQHandler                          0x00000263   Thumb Code     0  startup_k1921vk035.o(.text)
    CAN10_IRQHandler                         0x00000263   Thumb Code     0  startup_k1921vk035.o(.text)
    CAN11_IRQHandler                         0x00000263   Thumb Code     0  startup_k1921vk035.o(.text)
    CAN12_IRQHandler                         0x00000263   Thumb Code     0  startup_k1921vk035.o(.text)
    CAN13_IRQHandler                         0x00000263   Thumb Code     0  startup_k1921vk035.o(.text)
    CAN14_IRQHandler                         0x00000263   Thumb Code     0  startup_k1921vk035.o(.text)
    CAN15_IRQHandler                         0x00000263   Thumb Code     0  startup_k1921vk035.o(.text)
    CAN1_IRQHandler                          0x00000263   Thumb Code     0  startup_k1921vk035.o(.text)
    CAN2_IRQHandler                          0x00000263   Thumb Code     0  startup_k1921vk035.o(.text)
    CAN3_IRQHandler                          0x00000263   Thumb Code     0  startup_k1921vk035.o(.text)
    CAN4_IRQHandler                          0x00000263   Thumb Code     0  startup_k1921vk035.o(.text)
    CAN5_IRQHandler                          0x00000263   Thumb Code     0  startup_k1921vk035.o(.text)
    CAN6_IRQHandler                          0x00000263   Thumb Code     0  startup_k1921vk035.o(.text)
    CAN7_IRQHandler                          0x00000263   Thumb Code     0  startup_k1921vk035.o(.text)
    CAN8_IRQHandler                          0x00000263   Thumb Code     0  startup_k1921vk035.o(.text)
    CAN9_IRQHandler                          0x00000263   Thumb Code     0  startup_k1921vk035.o(.text)
    DMA_CH0_IRQHandler                       0x00000263   Thumb Code     0  startup_k1921vk035.o(.text)
    DMA_CH10_IRQHandler                      0x00000263   Thumb Code     0  startup_k1921vk035.o(.text)
    DMA_CH11_IRQHandler                      0x00000263   Thumb Code     0  startup_k1921vk035.o(.text)
    DMA_CH12_IRQHandler                      0x00000263   Thumb Code     0  startup_k1921vk035.o(.text)
    DMA_CH13_IRQHandler                      0x00000263   Thumb Code     0  startup_k1921vk035.o(.text)
    DMA_CH14_IRQHandler                      0x00000263   Thumb Code     0  startup_k1921vk035.o(.text)
    DMA_CH15_IRQHandler                      0x00000263   Thumb Code     0  startup_k1921vk035.o(.text)
    DMA_CH1_IRQHandler                       0x00000263   Thumb Code     0  startup_k1921vk035.o(.text)
    DMA_CH2_IRQHandler                       0x00000263   Thumb Code     0  startup_k1921vk035.o(.text)
    DMA_CH3_IRQHandler                       0x00000263   Thumb Code     0  startup_k1921vk035.o(.text)
    DMA_CH4_IRQHandler                       0x00000263   Thumb Code     0  startup_k1921vk035.o(.text)
    DMA_CH5_IRQHandler                       0x00000263   Thumb Code     0  startup_k1921vk035.o(.text)
    DMA_CH6_IRQHandler                       0x00000263   Thumb Code     0  startup_k1921vk035.o(.text)
    DMA_CH7_IRQHandler                       0x00000263   Thumb Code     0  startup_k1921vk035.o(.text)
    DMA_CH8_IRQHandler                       0x00000263   Thumb Code     0  startup_k1921vk035.o(.text)
    DMA_CH9_IRQHandler                       0x00000263   Thumb Code     0  startup_k1921vk035.o(.text)
    ECAP0_IRQHandler                         0x00000263   Thumb Code     0  startup_k1921vk035.o(.text)
    ECAP1_IRQHandler                         0x00000263   Thumb Code     0  startup_k1921vk035.o(.text)
    ECAP2_IRQHandler                         0x00000263   Thumb Code     0  startup_k1921vk035.o(.text)
    FPU_IRQHandler                           0x00000263   Thumb Code     0  startup_k1921vk035.o(.text)
    GPIOA_IRQHandler                         0x00000263   Thumb Code     0  startup_k1921vk035.o(.text)
    GPIOB_IRQHandler                         0x00000263   Thumb Code     0  startup_k1921vk035.o(.text)
    I2C_IRQHandler                           0x00000263   Thumb Code     0  startup_k1921vk035.o(.text)
    MFLASH_IRQHandler                        0x00000263   Thumb Code     0  startup_k1921vk035.o(.text)
    PWM0_HD_IRQHandler                       0x00000263   Thumb Code     0  startup_k1921vk035.o(.text)
    PWM0_IRQHandler                          0x00000263   Thumb Code     0  startup_k1921vk035.o(.text)
    PWM0_TZ_IRQHandler                       0x00000263   Thumb Code     0  startup_k1921vk035.o(.text)
    PWM1_HD_IRQHandler                       0x00000263   Thumb Code     0  startup_k1921vk035.o(.text)
    PWM1_IRQHandler                          0x00000263   Thumb Code     0  startup_k1921vk035.o(.text)
    PWM1_TZ_IRQHandler                       0x00000263   Thumb Code     0  startup_k1921vk035.o(.text)
    PWM2_HD_IRQHandler                       0x00000263   Thumb Code     0  startup_k1921vk035.o(.text)
    PWM2_IRQHandler                          0x00000263   Thumb Code     0  startup_k1921vk035.o(.text)
    PWM2_TZ_IRQHandler                       0x00000263   Thumb Code     0  startup_k1921vk035.o(.text)
    QEP_IRQHandler                           0x00000263   Thumb Code     0  startup_k1921vk035.o(.text)
    RCU_IRQHandler                           0x00000263   Thumb Code     0  startup_k1921vk035.o(.text)
    SPI_RO_RT_IRQHandler                     0x00000263   Thumb Code     0  startup_k1921vk035.o(.text)
    SPI_RX_IRQHandler                        0x00000263   Thumb Code     0  startup_k1921vk035.o(.text)
    SPI_TX_IRQHandler                        0x00000263   Thumb Code     0  startup_k1921vk035.o(.text)
    TMR0_IRQHandler                          0x00000263   Thumb Code     0  startup_k1921vk035.o(.text)
    TMR1_IRQHandler                          0x00000263   Thumb Code     0  startup_k1921vk035.o(.text)
    TMR2_IRQHandler                          0x00000263   Thumb Code     0  startup_k1921vk035.o(.text)
    TMR3_IRQHandler                          0x00000263   Thumb Code     0  startup_k1921vk035.o(.text)
    UART0_E_RT_IRQHandler                    0x00000263   Thumb Code     0  startup_k1921vk035.o(.text)
    UART0_RX_IRQHandler                      0x00000263   Thumb Code     0  startup_k1921vk035.o(.text)
    UART0_TD_IRQHandler                      0x00000263   Thumb Code     0  startup_k1921vk035.o(.text)
    UART0_TX_IRQHandler                      0x00000263   Thumb Code     0  startup_k1921vk035.o(.text)
    UART1_E_RT_IRQHandler                    0x00000263   Thumb Code     0  startup_k1921vk035.o(.text)
    UART1_RX_IRQHandler                      0x00000263   Thumb Code     0  startup_k1921vk035.o(.text)
    UART1_TD_IRQHandler                      0x00000263   Thumb Code     0  startup_k1921vk035.o(.text)
    UART1_TX_IRQHandler                      0x00000263   Thumb Code     0  startup_k1921vk035.o(.text)
    WDT_IRQHandler                           0x00000263   Thumb Code     0  startup_k1921vk035.o(.text)
    __user_initial_stackheap                 0x00000265   Thumb Code     0  startup_k1921vk035.o(.text)
    __I$use$semihosting                      0x00000289   Thumb Code     0  use_no_semi.o(.text)
    __use_no_semihosting_swi                 0x00000289   Thumb Code     2  use_no_semi.o(.text)
    __2printf                                0x0000028d   Thumb Code    20  noretval__2printf.o(.text)
    _printf_pre_padding                      0x000002a5   Thumb Code    44  _printf_pad.o(.text)
    _printf_post_padding                     0x000002d1   Thumb Code    34  _printf_pad.o(.text)
    _printf_str                              0x000002f3   Thumb Code    82  _printf_str.o(.text)
    _printf_int_dec                          0x00000345   Thumb Code   104  _printf_dec.o(.text)
    __printf                                 0x000003bd   Thumb Code   270  __printf_wp.o(.text)
    __use_two_region_memory                  0x000004cb   Thumb Code     2  heapauxi.o(.text)
    __rt_heap_escrow$2region                 0x000004cd   Thumb Code     2  heapauxi.o(.text)
    __rt_heap_expand$2region                 0x000004cf   Thumb Code     2  heapauxi.o(.text)
    _printf_int_common                       0x000004d1   Thumb Code   178  _printf_intcommon.o(.text)
    _printf_cs_common                        0x00000583   Thumb Code    20  _printf_char.o(.text)
    _printf_char                             0x00000597   Thumb Code    16  _printf_char.o(.text)
    _printf_string                           0x000005a7   Thumb Code     8  _printf_char.o(.text)
    _printf_char_file                        0x000005b1   Thumb Code    32  _printf_char_file.o(.text)
    _printf_char_common                      0x000005df   Thumb Code    32  _printf_char_common.o(.text)
    __user_setup_stackheap                   0x00000605   Thumb Code    74  sys_stackheap_outer.o(.text)
    exit                                     0x0000064f   Thumb Code    18  exit.o(.text)
    __user_libspace                          0x00000661   Thumb Code     8  libspace.o(.text)
    __user_perproc_libspace                  0x00000661   Thumb Code     0  libspace.o(.text)
    __user_perthread_libspace                0x00000661   Thumb Code     0  libspace.o(.text)
    BusFault_Handler                         0x00000669   Thumb Code     2  vk035_it.o(i.BusFault_Handler)
    ClkInit                                  0x0000066d   Thumb Code   106  system_k1921vk035.o(i.ClkInit)
    DebugMon_Handler                         0x000006e1   Thumb Code     2  vk035_it.o(i.DebugMon_Handler)
    Error_Handler                            0x000006e3   Thumb Code     4  main.o(i.Error_Handler)
    FPUInit                                  0x000006e9   Thumb Code    18  system_k1921vk035.o(i.FPUInit)
    GPIO_DeInit                              0x00000759   Thumb Code    54  plib035_gpio.o(i.GPIO_DeInit)
    GPIO_DriveModeConfig                     0x00000839   Thumb Code    80  plib035_gpio.o(i.GPIO_DriveModeConfig)
    GPIO_InModeConfig                        0x000008b5   Thumb Code    76  plib035_gpio.o(i.GPIO_InModeConfig)
    GPIO_Init                                0x0000092d   Thumb Code    80  plib035_gpio.o(i.GPIO_Init)
    GPIO_OutModeConfig                       0x00000a01   Thumb Code    76  plib035_gpio.o(i.GPIO_OutModeConfig)
    GPIO_PullModeConfig                      0x00000a79   Thumb Code    76  plib035_gpio.o(i.GPIO_PullModeConfig)
    HardFault_Handler                        0x00000af1   Thumb Code     2  vk035_it.o(i.HardFault_Handler)
    MemManage_Handler                        0x00000b3d   Thumb Code     2  vk035_it.o(i.MemManage_Handler)
    NMI_Handler                              0x00000b3f   Thumb Code     2  vk035_it.o(i.NMI_Handler)
    PendSV_Handler                           0x00000b41   Thumb Code     2  vk035_it.o(i.PendSV_Handler)
    RCU_PLL_AutoConfig                       0x00000c39   Thumb Code   304  plib035_rcu.o(i.RCU_PLL_AutoConfig)
    RCU_PLL_Init                             0x00000d99   Thumb Code   212  plib035_rcu.o(i.RCU_PLL_Init)
    RCU_PLL_StructInit                       0x00000ee9   Thumb Code    16  plib035_rcu.o(i.RCU_PLL_StructInit)
    RCU_SysClkChangeCmd                      0x00000ef9   Thumb Code   104  plib035_rcu.o(i.RCU_SysClkChangeCmd)
    SVC_Handler                              0x00000fb1   Thumb Code     2  vk035_it.o(i.SVC_Handler)
    SysTick_Handler                          0x00000fb5   Thumb Code    10  vk035_it.o(i.SysTick_Handler)
    SystemCoreClockUpdate                    0x00000fc5   Thumb Code    96  system_k1921vk035.o(i.SystemCoreClockUpdate)
    SystemInit                               0x00001035   Thumb Code    14  system_k1921vk035.o(i.SystemInit)
    UsageFault_Handler                       0x00001043   Thumb Code     2  vk035_it.o(i.UsageFault_Handler)
    _is_digit                                0x00001045   Thumb Code    14  __printf_wp.o(i._is_digit)
    _sys_exit                                0x00001053   Thumb Code     2  retarget.o(i._sys_exit)
    assert_failed                            0x00001055   Thumb Code    12  main.o(i.assert_failed)
    ferror                                   0x00001085   Thumb Code     6  retarget.o(i.ferror)
    fputc                                    0x0000108b   Thumb Code     4  retarget.o(i.fputc)
    gpio_init                                0x00001091   Thumb Code   100  gpio.o(i.gpio_init)
    main                                     0x00001105   Thumb Code     6  main.o(i.main)
    periph_init                              0x0000110d   Thumb Code    54  main.o(i.periph_init)
    retarget_init                            0x0000117d   Thumb Code   166  retarget_conf.o(i.retarget_init)
    retarget_put_char                        0x0000123d   Thumb Code    14  retarget_conf.o(i.retarget_put_char)
    sysclk_init                              0x00001251   Thumb Code    80  rcu.o(i.sysclk_init)
    __aeabi_ddiv                             0x000012b9   Thumb Code     0  ddiv.o(x$fpl$ddiv)
    _ddiv                                    0x000012b9   Thumb Code   552  ddiv.o(x$fpl$ddiv)
    __aeabi_d2iz                             0x00001569   Thumb Code     0  dfix.o(x$fpl$dfix)
    _dfix                                    0x00001569   Thumb Code    94  dfix.o(x$fpl$dfix)
    __aeabi_ui2d                             0x000015c7   Thumb Code     0  dflt_clz.o(x$fpl$dfltu)
    _dfltu                                   0x000015c7   Thumb Code    38  dflt_clz.o(x$fpl$dfltu)
    __fpl_dnaninf                            0x000015ed   Thumb Code   156  dnaninf.o(x$fpl$dnaninf)
    __fpl_dretinf                            0x00001689   Thumb Code    12  dretinf.o(x$fpl$dretinf)
    _fp_init                                 0x00001695   Thumb Code    10  fpinit.o(x$fpl$fpinit)
    __fplib_config_fpu_vfp                   0x0000169d   Thumb Code     0  fpinit.o(x$fpl$fpinit)
    __fplib_config_pureend_doubles           0x0000169d   Thumb Code     0  fpinit.o(x$fpl$fpinit)
    __I$use$fp                               0x0000169e   Number         0  usenofp.o(x$fpl$usenofp)
    Region$$Table$$Base                      0x000016a0   Number         0  anon$$obj.o(Region$$Table)
    Region$$Table$$Limit                     0x000016c0   Number         0  anon$$obj.o(Region$$Table)
    SystemCoreClock                          0x20000000   Data           4  system_k1921vk035.o(.data)
    uwTick                                   0x20000004   Data           4  system_k1921vk035.o(.data)
    __stdout                                 0x2000018c   Data           4  retarget.o(.data)
    __libspace_start                         0x20000190   Data          96  libspace.o(.bss)
    __temporary_stack_top$libspace           0x200001f0   Data           0  libspace.o(.bss)



==============================================================================

Memory Map of the image

  Image Entry point : 0x00000249

  Load Region LR_1 (Base: 0x00000000, Size: 0x00001850, Max: 0xffffffff, ABSOLUTE, COMPRESSED[0x000016e4])

    Execution Region ER_RO (Exec base: 0x00000000, Load base: 0x00000000, Size: 0x000016c0, Max: 0xffffffff, ABSOLUTE)

    Exec Addr    Load Addr    Size         Type   Attr      Idx    E Section Name        Object

    0x00000000   0x00000000   0x00000158   Data   RO           77    RESET               startup_k1921vk035.o
    0x00000158   0x00000158   0x00000008   Code   RO         1417  * !!!main             c_w.l(__main.o)
    0x00000160   0x00000160   0x00000034   Code   RO         1602    !!!scatter          c_w.l(__scatter.o)
    0x00000194   0x00000194   0x0000005a   Code   RO         1600    !!dczerorl2         c_w.l(__dczerorl2.o)
    0x000001ee   0x000001ee   0x00000002   PAD
    0x000001f0   0x000001f0   0x0000001c   Code   RO         1604    !!handler_zi        c_w.l(__scatter_zi.o)
    0x0000020c   0x0000020c   0x00000000   Code   RO         1414    .ARM.Collect$$_printf_percent$$00000000  c_w.l(_printf_percent.o)
    0x0000020c   0x0000020c   0x00000006   Code   RO         1413    .ARM.Collect$$_printf_percent$$00000009  c_w.l(_printf_d.o)
    0x00000212   0x00000212   0x00000006   Code   RO         1412    .ARM.Collect$$_printf_percent$$00000014  c_w.l(_printf_s.o)
    0x00000218   0x00000218   0x00000004   Code   RO         1440    .ARM.Collect$$_printf_percent$$00000017  c_w.l(_printf_percent_end.o)
    0x0000021c   0x0000021c   0x00000002   Code   RO         1474    .ARM.Collect$$libinit$$00000000  c_w.l(libinit.o)
    0x0000021e   0x0000021e   0x00000004   Code   RO         1480    .ARM.Collect$$libinit$$00000001  c_w.l(libinit2.o)
    0x00000222   0x00000222   0x00000000   Code   RO         1483    .ARM.Collect$$libinit$$00000004  c_w.l(libinit2.o)
    0x00000222   0x00000222   0x00000000   Code   RO         1486    .ARM.Collect$$libinit$$0000000A  c_w.l(libinit2.o)
    0x00000222   0x00000222   0x00000000   Code   RO         1488    .ARM.Collect$$libinit$$0000000C  c_w.l(libinit2.o)
    0x00000222   0x00000222   0x00000000   Code   RO         1490    .ARM.Collect$$libinit$$0000000E  c_w.l(libinit2.o)
    0x00000222   0x00000222   0x00000000   Code   RO         1493    .ARM.Collect$$libinit$$00000011  c_w.l(libinit2.o)
    0x00000222   0x00000222   0x00000000   Code   RO         1495    .ARM.Collect$$libinit$$00000013  c_w.l(libinit2.o)
    0x00000222   0x00000222   0x00000000   Code   RO         1497    .ARM.Collect$$libinit$$00000015  c_w.l(libinit2.o)
    0x00000222   0x00000222   0x00000000   Code   RO         1499    .ARM.Collect$$libinit$$00000017  c_w.l(libinit2.o)
    0x00000222   0x00000222   0x00000000   Code   RO         1501    .ARM.Collect$$libinit$$00000019  c_w.l(libinit2.o)
    0x00000222   0x00000222   0x00000000   Code   RO         1503    .ARM.Collect$$libinit$$0000001B  c_w.l(libinit2.o)
    0x00000222   0x00000222   0x00000000   Code   RO         1505    .ARM.Collect$$libinit$$0000001D  c_w.l(libinit2.o)
    0x00000222   0x00000222   0x00000000   Code   RO         1507    .ARM.Collect$$libinit$$0000001F  c_w.l(libinit2.o)
    0x00000222   0x00000222   0x00000000   Code   RO         1509    .ARM.Collect$$libinit$$00000021  c_w.l(libinit2.o)
    0x00000222   0x00000222   0x00000000   Code   RO         1511    .ARM.Collect$$libinit$$00000023  c_w.l(libinit2.o)
    0x00000222   0x00000222   0x00000000   Code   RO         1513    .ARM.Collect$$libinit$$00000025  c_w.l(libinit2.o)
    0x00000222   0x00000222   0x00000000   Code   RO         1517    .ARM.Collect$$libinit$$0000002C  c_w.l(libinit2.o)
    0x00000222   0x00000222   0x00000000   Code   RO         1519    .ARM.Collect$$libinit$$0000002E  c_w.l(libinit2.o)
    0x00000222   0x00000222   0x00000000   Code   RO         1521    .ARM.Collect$$libinit$$00000030  c_w.l(libinit2.o)
    0x00000222   0x00000222   0x00000000   Code   RO         1523    .ARM.Collect$$libinit$$00000032  c_w.l(libinit2.o)
    0x00000222   0x00000222   0x00000002   Code   RO         1524    .ARM.Collect$$libinit$$00000033  c_w.l(libinit2.o)
    0x00000224   0x00000224   0x00000002   Code   RO         1542    .ARM.Collect$$libshutdown$$00000000  c_w.l(libshutdown.o)
    0x00000226   0x00000226   0x00000000   Code   RO         1552    .ARM.Collect$$libshutdown$$00000002  c_w.l(libshutdown2.o)
    0x00000226   0x00000226   0x00000000   Code   RO         1554    .ARM.Collect$$libshutdown$$00000004  c_w.l(libshutdown2.o)
    0x00000226   0x00000226   0x00000000   Code   RO         1556    .ARM.Collect$$libshutdown$$00000006  c_w.l(libshutdown2.o)
    0x00000226   0x00000226   0x00000000   Code   RO         1559    .ARM.Collect$$libshutdown$$00000009  c_w.l(libshutdown2.o)
    0x00000226   0x00000226   0x00000000   Code   RO         1562    .ARM.Collect$$libshutdown$$0000000C  c_w.l(libshutdown2.o)
    0x00000226   0x00000226   0x00000000   Code   RO         1564    .ARM.Collect$$libshutdown$$0000000E  c_w.l(libshutdown2.o)
    0x00000226   0x00000226   0x00000000   Code   RO         1567    .ARM.Collect$$libshutdown$$00000011  c_w.l(libshutdown2.o)
    0x00000226   0x00000226   0x00000002   Code   RO         1568    .ARM.Collect$$libshutdown$$00000012  c_w.l(libshutdown2.o)
    0x00000228   0x00000228   0x00000000   Code   RO         1433    .ARM.Collect$$rtentry$$00000000  c_w.l(__rtentry.o)
    0x00000228   0x00000228   0x00000000   Code   RO         1447    .ARM.Collect$$rtentry$$00000002  c_w.l(__rtentry2.o)
    0x00000228   0x00000228   0x00000006   Code   RO         1459    .ARM.Collect$$rtentry$$00000004  c_w.l(__rtentry4.o)
    0x0000022e   0x0000022e   0x00000000   Code   RO         1449    .ARM.Collect$$rtentry$$00000009  c_w.l(__rtentry2.o)
    0x0000022e   0x0000022e   0x00000004   Code   RO         1450    .ARM.Collect$$rtentry$$0000000A  c_w.l(__rtentry2.o)
    0x00000232   0x00000232   0x00000000   Code   RO         1452    .ARM.Collect$$rtentry$$0000000C  c_w.l(__rtentry2.o)
    0x00000232   0x00000232   0x00000008   Code   RO         1453    .ARM.Collect$$rtentry$$0000000D  c_w.l(__rtentry2.o)
    0x0000023a   0x0000023a   0x00000002   Code   RO         1478    .ARM.Collect$$rtexit$$00000000  c_w.l(rtexit.o)
    0x0000023c   0x0000023c   0x00000000   Code   RO         1526    .ARM.Collect$$rtexit$$00000002  c_w.l(rtexit2.o)
    0x0000023c   0x0000023c   0x00000004   Code   RO         1527    .ARM.Collect$$rtexit$$00000003  c_w.l(rtexit2.o)
    0x00000240   0x00000240   0x00000006   Code   RO         1528    .ARM.Collect$$rtexit$$00000004  c_w.l(rtexit2.o)
    0x00000246   0x00000246   0x00000002   PAD
    0x00000248   0x00000248   0x00000040   Code   RO           78  * .text               startup_k1921vk035.o
    0x00000288   0x00000288   0x00000002   Code   RO         1378    .text               c_w.l(use_no_semi.o)
    0x0000028a   0x0000028a   0x00000002   PAD
    0x0000028c   0x0000028c   0x00000018   Code   RO         1382    .text               c_w.l(noretval__2printf.o)
    0x000002a4   0x000002a4   0x0000004e   Code   RO         1386    .text               c_w.l(_printf_pad.o)
    0x000002f2   0x000002f2   0x00000052   Code   RO         1388    .text               c_w.l(_printf_str.o)
    0x00000344   0x00000344   0x00000078   Code   RO         1390    .text               c_w.l(_printf_dec.o)
    0x000003bc   0x000003bc   0x0000010e   Code   RO         1400    .text               c_w.l(__printf_wp.o)
    0x000004ca   0x000004ca   0x00000006   Code   RO         1415    .text               c_w.l(heapauxi.o)
    0x000004d0   0x000004d0   0x000000b2   Code   RO         1434    .text               c_w.l(_printf_intcommon.o)
    0x00000582   0x00000582   0x0000002c   Code   RO         1436    .text               c_w.l(_printf_char.o)
    0x000005ae   0x000005ae   0x00000002   PAD
    0x000005b0   0x000005b0   0x00000024   Code   RO         1438    .text               c_w.l(_printf_char_file.o)
    0x000005d4   0x000005d4   0x00000030   Code   RO         1461    .text               c_w.l(_printf_char_common.o)
    0x00000604   0x00000604   0x0000004a   Code   RO         1463    .text               c_w.l(sys_stackheap_outer.o)
    0x0000064e   0x0000064e   0x00000012   Code   RO         1467    .text               c_w.l(exit.o)
    0x00000660   0x00000660   0x00000008   Code   RO         1475    .text               c_w.l(libspace.o)
    0x00000668   0x00000668   0x00000002   Code   RO          274    i.BusFault_Handler  vk035_it.o
    0x0000066a   0x0000066a   0x00000002   PAD
    0x0000066c   0x0000066c   0x00000074   Code   RO            4    i.ClkInit           system_k1921vk035.o
    0x000006e0   0x000006e0   0x00000002   Code   RO          275    i.DebugMon_Handler  vk035_it.o
    0x000006e2   0x000006e2   0x00000004   Code   RO           85    i.Error_Handler     main.o
    0x000006e6   0x000006e6   0x00000002   PAD
    0x000006e8   0x000006e8   0x00000018   Code   RO            5    i.FPUInit           system_k1921vk035.o
    0x00000700   0x00000700   0x00000058   Code   RO          571    i.GPIO_AltFuncCmd   plib035_gpio.o
    0x00000758   0x00000758   0x00000064   Code   RO          572    i.GPIO_DeInit       plib035_gpio.o
    0x000007bc   0x000007bc   0x0000007c   Code   RO          573    i.GPIO_DigitalCmd   plib035_gpio.o
    0x00000838   0x00000838   0x0000007c   Code   RO          574    i.GPIO_DriveModeConfig  plib035_gpio.o
    0x000008b4   0x000008b4   0x00000078   Code   RO          575    i.GPIO_InModeConfig  plib035_gpio.o
    0x0000092c   0x0000092c   0x00000050   Code   RO          576    i.GPIO_Init         plib035_gpio.o
    0x0000097c   0x0000097c   0x0000002c   Code   RO          577    i.GPIO_ModeConfig   plib035_gpio.o
    0x000009a8   0x000009a8   0x00000058   Code   RO          578    i.GPIO_OutCmd       plib035_gpio.o
    0x00000a00   0x00000a00   0x00000078   Code   RO          579    i.GPIO_OutModeConfig  plib035_gpio.o
    0x00000a78   0x00000a78   0x00000078   Code   RO          580    i.GPIO_PullModeConfig  plib035_gpio.o
    0x00000af0   0x00000af0   0x00000002   Code   RO          276    i.HardFault_Handler  vk035_it.o
    0x00000af2   0x00000af2   0x00000002   PAD
    0x00000af4   0x00000af4   0x00000048   Code   RO          977    i.MFLASH_LatencyConfig  plib035_rcu.o
    0x00000b3c   0x00000b3c   0x00000002   Code   RO          277    i.MemManage_Handler  vk035_it.o
    0x00000b3e   0x00000b3e   0x00000002   Code   RO          278    i.NMI_Handler       vk035_it.o
    0x00000b40   0x00000b40   0x00000002   Code   RO          279    i.PendSV_Handler    vk035_it.o
    0x00000b42   0x00000b42   0x00000002   PAD
    0x00000b44   0x00000b44   0x0000006c   Code   RO          582    i.RCU_AHBRstCmd     plib035_gpio.o
    0x00000bb0   0x00000bb0   0x00000088   Code   RO          236    i.RCU_ClkOutConfig  rcu.o
    0x00000c38   0x00000c38   0x00000160   Code   RO          989    i.RCU_PLL_AutoConfig  plib035_rcu.o
    0x00000d98   0x00000d98   0x00000100   Code   RO          991    i.RCU_PLL_Init      plib035_rcu.o
    0x00000e98   0x00000e98   0x00000050   Code   RO          992    i.RCU_PLL_OutCmd    plib035_rcu.o
    0x00000ee8   0x00000ee8   0x00000010   Code   RO          993    i.RCU_PLL_StructInit  plib035_rcu.o
    0x00000ef8   0x00000ef8   0x000000b8   Code   RO          994    i.RCU_SysClkChangeCmd  plib035_rcu.o
    0x00000fb0   0x00000fb0   0x00000002   Code   RO          280    i.SVC_Handler       vk035_it.o
    0x00000fb2   0x00000fb2   0x00000002   PAD
    0x00000fb4   0x00000fb4   0x00000010   Code   RO          281    i.SysTick_Handler   vk035_it.o
    0x00000fc4   0x00000fc4   0x00000070   Code   RO            6    i.SystemCoreClockUpdate  system_k1921vk035.o
    0x00001034   0x00001034   0x0000000e   Code   RO            7    i.SystemInit        system_k1921vk035.o
    0x00001042   0x00001042   0x00000002   Code   RO          282    i.UsageFault_Handler  vk035_it.o
    0x00001044   0x00001044   0x0000000e   Code   RO         1402    i._is_digit         c_w.l(__printf_wp.o)
    0x00001052   0x00001052   0x00000002   Code   RO         1278    i._sys_exit         retarget.o
    0x00001054   0x00001054   0x00000030   Code   RO           86    i.assert_failed     main.o
    0x00001084   0x00001084   0x00000006   Code   RO         1280    i.ferror            retarget.o
    0x0000108a   0x0000108a   0x00000004   Code   RO         1282    i.fputc             retarget.o
    0x0000108e   0x0000108e   0x00000002   PAD
    0x00001090   0x00001090   0x00000074   Code   RO          204    i.gpio_init         gpio.o
    0x00001104   0x00001104   0x00000006   Code   RO           87    i.main              main.o
    0x0000110a   0x0000110a   0x00000002   PAD
    0x0000110c   0x0000110c   0x00000070   Code   RO           88    i.periph_init       main.o
    0x0000117c   0x0000117c   0x000000c0   Code   RO         1344    i.retarget_init     retarget_conf.o
    0x0000123c   0x0000123c   0x00000014   Code   RO         1345    i.retarget_put_char  retarget_conf.o
    0x00001250   0x00001250   0x00000068   Code   RO          237    i.sysclk_init       rcu.o
    0x000012b8   0x000012b8   0x000002b0   Code   RO         1420    x$fpl$ddiv          fz_wm.l(ddiv.o)
    0x00001568   0x00001568   0x0000005e   Code   RO         1423    x$fpl$dfix          fz_wm.l(dfix.o)
    0x000015c6   0x000015c6   0x00000026   Code   RO         1427    x$fpl$dfltu         fz_wm.l(dflt_clz.o)
    0x000015ec   0x000015ec   0x0000009c   Code   RO         1441    x$fpl$dnaninf       fz_wm.l(dnaninf.o)
    0x00001688   0x00001688   0x0000000c   Code   RO         1443    x$fpl$dretinf       fz_wm.l(dretinf.o)
    0x00001694   0x00001694   0x0000000a   Code   RO         1534    x$fpl$fpinit        fz_wm.l(fpinit.o)
    0x0000169e   0x0000169e   0x00000000   Code   RO         1445    x$fpl$usenofp       fz_wm.l(usenofp.o)
    0x0000169e   0x0000169e   0x00000002   PAD
    0x000016a0   0x000016a0   0x00000020   Data   RO         1598    Region$$Table       anon$$obj.o


    Execution Region ER_RW (Exec base: 0x20000000, Load base: 0x000016c0, Size: 0x00000190, Max: 0xffffffff, ABSOLUTE, COMPRESSED[0x00000024])

    Exec Addr    Load Addr    Size         Type   Attr      Idx    E Section Name        Object

    0x20000000   COMPRESSED   0x00000004   Data   RW            8    .data               system_k1921vk035.o
    0x20000004   COMPRESSED   0x00000004   Data   RW            9    .data               system_k1921vk035.o
    0x20000008   COMPRESSED   0x00000180   Data   RW          205    .data               gpio.o
    0x20000188   COMPRESSED   0x00000001   Data   RW          238    .data               rcu.o
    0x20000189   COMPRESSED   0x00000003   PAD
    0x2000018c   COMPRESSED   0x00000004   Data   RW         1283    .data               retarget.o


    Execution Region ER_ZI (Exec base: 0x20000190, Load base: 0x000016e4, Size: 0x00000660, Max: 0xffffffff, ABSOLUTE)

    Exec Addr    Load Addr    Size         Type   Attr      Idx    E Section Name        Object

    0x20000190        -       0x00000060   Zero   RW         1476    .bss                c_w.l(libspace.o)
    0x200001f0        -       0x00000200   Zero   RW           76    HEAP                startup_k1921vk035.o
    0x200003f0        -       0x00000400   Zero   RW           75    STACK               startup_k1921vk035.o


==============================================================================

Image component sizes


      Code (inc. data)   RO Data    RW Data    ZI Data      Debug   Object Name

       116         16          0        384          0      10416   gpio.o
       170         94          0          0          0       8505   main.o
      1116        344          0          0          0      12904   plib035_gpio.o
       960        262          0          0          0      15871   plib035_rcu.o
       240         74          0          1          0      40297   rcu.o
        12          0          0          4          0       3303   retarget.o
       212         32          0          0          0       1204   retarget_conf.o
        64         26        344          0       1536        892   startup_k1921vk035.o
       266         32          0          8          0     197926   system_k1921vk035.o
        32          6          0          0          0       3974   vk035_it.o

    ----------------------------------------------------------------------
      3202        886        376        400       1536     295292   Object Totals
         0          0         32          0          0          0   (incl. Generated)
        14          0          0          3          0          0   (incl. Padding)

    ----------------------------------------------------------------------

      Code (inc. data)   RO Data    RW Data    ZI Data      Debug   Library Member Name

        90          0          0          0          0          0   __dczerorl2.o
         8          0          0          0          0         68   __main.o
       284          0          0          0          0        156   __printf_wp.o
         0          0          0          0          0          0   __rtentry.o
        12          0          0          0          0          0   __rtentry2.o
         6          0          0          0          0          0   __rtentry4.o
        52          8          0          0          0          0   __scatter.o
        28          0          0          0          0          0   __scatter_zi.o
        44          0          0          0          0        108   _printf_char.o
        48          6          0          0          0         96   _printf_char_common.o
        36          4          0          0          0         80   _printf_char_file.o
         6          0          0          0          0          0   _printf_d.o
       120         16          0          0          0         92   _printf_dec.o
       178          0          0          0          0         88   _printf_intcommon.o
        78          0          0          0          0        108   _printf_pad.o
         0          0          0          0          0          0   _printf_percent.o
         4          0          0          0          0          0   _printf_percent_end.o
         6          0          0          0          0          0   _printf_s.o
        82          0          0          0          0         80   _printf_str.o
        18          0          0          0          0         80   exit.o
         6          0          0          0          0        152   heapauxi.o
         2          0          0          0          0          0   libinit.o
         6          0          0          0          0          0   libinit2.o
         2          0          0          0          0          0   libshutdown.o
         2          0          0          0          0          0   libshutdown2.o
         8          4          0          0         96         68   libspace.o
        24          4          0          0          0         84   noretval__2printf.o
         2          0          0          0          0          0   rtexit.o
        10          0          0          0          0          0   rtexit2.o
        74          0          0          0          0         80   sys_stackheap_outer.o
         2          0          0          0          0         68   use_no_semi.o
       688        140          0          0          0        256   ddiv.o
        94          4          0          0          0        140   dfix.o
        38          0          0          0          0        116   dflt_clz.o
       156          4          0          0          0        140   dnaninf.o
        12          0          0          0          0        116   dretinf.o
        10          0          0          0          0        116   fpinit.o
         0          0          0          0          0          0   usenofp.o

    ----------------------------------------------------------------------
      2246        190          0          0         96       2292   Library Totals
        10          0          0          0          0          0   (incl. Padding)

    ----------------------------------------------------------------------

      Code (inc. data)   RO Data    RW Data    ZI Data      Debug   Library Name

      1238         42          0          0         96       1408   c_w.l
       998        148          0          0          0        884   fz_wm.l

    ----------------------------------------------------------------------
      2246        190          0          0         96       2292   Library Totals

    ----------------------------------------------------------------------

==============================================================================


      Code (inc. data)   RO Data    RW Data    ZI Data      Debug   

      5448       1076        376        400       1632     292960   Grand Totals
      5448       1076        376         36       1632     292960   ELF Image Totals (compressed)
      5448       1076        376         36          0          0   ROM Totals

==============================================================================

    Total RO  Size (Code + RO Data)                 5824 (   5.69kB)
    Total RW  Size (RW Data + ZI Data)              2032 (   1.98kB)
    Total ROM Size (Code + RO Data + RW Data)       5860 (   5.72kB)

==============================================================================

